S02B0000433A2F55736572732F766F6F72627572672F4465736B746F702F426C74546573742F546172676574E1
S31508000000003F0020890100083143000831430008F9
S3150800001031430008314300083143000831430008E2
S3150800002031430008314300083143000831430008D2
S3150800003031430008314300083143000831430008C2
S3150800004031430008314300083143000831430008B2
S3150800005031430008314300083143000831430008A2
S315080000603143000831430008314300083143000892
S315080000703143000831430008314300083143000882
S315080000803143000831430008314300083143000872
S315080000903143000831430008314300083143000862
S315080000A03143000831430008314300083143000852
S315080000B03143000831430008314300083143000842
S315080000C03143000831430008314300083143000832
S315080000D03143000831430008314300083143000822
S315080000E03143000831430008314300083143000812
S315080000F03143000831430008314300083143000802
S3150800010031430008314300083143000831430008F1
S3150800011031430008314300083143000831430008E1
S3150800012031430008314300083143000831430008D1
S3150800013031430008314300083143000831430008C1
S3150800014031430008314300083143000831430008B1
S3150800015031430008314300083143000831430008A1
S315080001603143000831430008314300083143000891
S315080001703143000831430008314300083143000881
S30D08000180314300083143000871
S315080001882949072291438D4628482949294A00F0D2
S3150800019839F8294829492A4A00F034F829482A49C1
S315080001A82A4A00F02FF82A482A492B4A00F02AF842
S315080001B82A482B492B4A00F025F82B482B492C4A64
S315080001C800F020F82B482C49002200F026F82B4886
S315080001D82B49091A082903DB00220260043001604A
S315080001E81C481D49884205D00268043003B4904764
S315080001F803BCF7E700208646EC4600200021214A82
S315080002089047FEE7884207D0521A05D0037801308E
S315080002180B700131013AF9D17047884202D0027051
S315080002280130FAE770470000003F00207CAE00085E
S3150800023800000020E500002090020008900200084F
S31508000248F8A300087CAE0008000000200000002083
S31508000258F8A30008F8A30008F8A30008F8A30008FC
S31508000268F8A30008F8A30008F8A30008F8A30008EC
S315080002787CAE0008E8000020002F0020002F002090
S30D0800028800370020593F000869
S3150800029010B54FF43053C4F20103586B10F0450FF4
S315080002A0FBD043070DD410F0010405D140F2FF50EE
S315080002B001F03AFC204610BD012001F035FC012072
S315080002C010BD042001F030FC032010BD4FF430525D
S315080002D038B5C4F201020446536B13F0450FFBD040
S315080002E059070DD413F0010505D101F0D5FBA0423D
S315080002F00BD0102038BD012001F016FC012038BDB6
S31508000300042001F011FC032038BD40F2FF5001F033
S315080003100BFC284601F0C8FB4EF20801CFF6FF5148
S31508000320014029B1002805DB420005D5092038BD62
S31508000330084638BD1C2038BD830001D50A2038BDC3
S31508000340C10001D50B2038BD020101D50C2038BDEE
S31508000350430101D50D2038BDC10101D50E2038BD98
S31508000360020201D50F2038BD4302C2D4810201D54D
S31508000370112038BDC20201D5122038BD030301D5AC
S31508000380132038BD410301D5142038BD820301D599
S31508000390152038BDC30301D5162038BD010401D583
S315080003A0172038BD420401D5182038BD830401D56D
S315080003B0192038BD10F0080F0CBF00201A2038BDD0
S315080003C02DE9F04F054685B0002001F06DFB10F0D1
S315080003D0007303D00E2005B0BDE8F08F854C02935C
S315080003E04FF0100920464FF0080840274FF4806662
S315080003F00393E36084E80003A760266101F034FBF9
S315080004004846FFF763FF01460029E4D1DFF8EC917F
S31508000410E160D9F80020A76012044FF0370A204699
S3150800042084E80404266101F01FFB5046FFF74EFFDF
S315080004300346002BCFD1704A4FF0FF3182E8020104
S3150800044030219160104602214FF0010A1361D160F4
S31508000450C2F814A0019301F035FB019BA7604FF089
S31508000460330B204684E80808E360266101F0FCFAAD
S315080004705846FFF72BFF0028ADD14FF43056C4F28B
S31508000480010640F22A63776B3B4007469BBB4FF455
S31508000490001001F03FFBB8BB42F210780EE0716B1A
S315080004A040F22A630B404FF4001008F1FF3813BBE3
S315080004B001F030FBB0B9B8F1010833D0726B40F2E5
S315080004C02A6111404FF40010A9B901F023FB002856
S315080004D0E5D001F00FFB04AB03EB8702013742F8C6
S315080004E0080CDCE701F006FB04A901EB87030137DA
S315080004F043F8080CDFE7082001F00CFB48B1082098
S3150800050001F012FB042066E701F0F4FA5746029060
S31508000510C2E7022001F0FEFA30B1022001F004FB26
S31508000520022058E7042056E7202001F0F3FA20B10C
S31508000530202001F0F9FA06204DE74FF4007001F08B
S31508000540E9FA064628B14FF4007001F0EDFA0720E3
S3150800055041E740F2FF5001F0E7FA0298012D02BA8E
S315080005602AD0D00301D4252035E7D9F80070214DCB
S31508000570E6603B04372628464FF040084FF480676C
S3150800058084E84801276101F06FFA3046FFF79EFEBE
S31508000590014600297FF41FAF0624284629606C60AF
S315080005A0C5F80880E9602F6101F05EFA204605B0BB
S315080005B0BDE8F04FFFF78ABE5303D4D5D9F800300B
S315080005C00C4DE6601B04372628464FF040084FF4CA
S315080005D0806784E84801276101F046FA3046FFF74C
S315080005E075FE014600297FF4F6AE02220624284647
S315080005F02A60D4E7A0010020EC0000204401002076
S3150800060000B54FF4006083B00123C4F202004FF432
S3150800061000618DF8073001F01DF908B98DF807005B
S315080006209DF8070003B000BD2DE9F04F834B844DBC
S3150800063085B00024184676221C605C609C60DC60ED
S315080006401C611A758DF80F4001F0DEF9032001F0E0
S31508000650FDF9012001F0F4F94FF4806128462C6079
S315080006606C60AC60EC6029614FF4803401F0FCF9F1
S3150800067006E0802001F04EFA40B9013C00F0C08047
S31508000680802001F047FA013C0028F2D040F2FF50E2
S3150800069001F04AFA00208DF80F009DF80F3023B1BB
S315080006A09DF80F0005B0BDE8F08F082240244FF4EE
S315080006B0D57185E816004FF43054C4F20104604839
S315080006C0EB604FF480672F6101F0CEF9626B12F090
S315080006D0450F0ED14FF4803105E0626B013912F0F7
S315080006E0450F05D141B1626B013912F0450FF4D0BF
S315080006F011B112F0040775D0042001F015FA032091
S315080007008DF80F009DF80F30002B7BD14D4F01243B
S315080007103C604FF0804400234FF037094022484898
S31508000720EB6085E808024FF48063AA602B6101F04C
S315080007309BF94846FFF7CAFD8DF80F009DF80F7024
S31508000740002FADD144F0004A4AF480104FF43054DB
S315080007503B4E0190B846C4F201043948C5F80080FA
S315080007604FF0400A4FF4806BC5F80490C5F808A00E
S31508000770C5F80C80C5F810B001F076F93720FFF7F8
S31508000780A5FD8DF80F009DF80F30002B88D1019933
S315080007902B48316029227260C6F808A0F360C6F8B3
S315080007A010B001F061F9606B10F0450FFBD010F046
S315080007B0040B1FD0042001F0B7F903238DF80F307E
S315080007C09DF80F0000287FF46BAF01F06DF9013733
S315080007D000284FF6FF7128DB8F42BED11B238DF808
S315080007E00F305DE712F040008AD0402001F09CF9F6
S315080007F0384685E740F2FF5001F096F95B46DDE79B
S31508000800032048E740224FF48061002437260C482D
S31508000810AA60296185E85000EC6001F025F93046A8
S31508000820FFF754FD8DF80F0075E78F42D6D04200CA
S315080008307FF536AF03480222026031E72C0100201B
S31508000840A001002014010020F8B501F005F910B93F
S3150800085025242046F8BD4E4E3368042B52D04D4D04
S31508000860002102224FF480632846C02429606A606A
S31508000870AC60E9602B6101F0F7F8FFF709FD044663
S315080008800028E6D101F010F9434F3860042001F042
S315080008900BF97860082001F007F9B8600C2001F020
S315080008A003F93368F860012B2FD9062B2DD0022BBC
S315080008B02BD00121042BCCD0384C364821600A04B1
S315080008C0C02309212A6000244FF480626960AB6066
S315080008D0EC602A6101F0C8F8FFF7DAFC0446002844
S315080008E0B7D101F0E1F82E4D2860042001F0DCF8BC
S315080008F06860082001F0D8F8A8600C2001F0D4F848
S31508000900E860A6E700242046F8BD002121482960B2
S3150800091003224023E9604FF480616A60AB60296175
S3150800092001F0A2F84FF43050C4F20100426B12F005
S31508000930450FFBD0500708D412F001070AD101F081
S31508000940ABF803280BD0102483E7042001F0ECF859
S3150800095003247EE7012001F0E7F8012479E740F255
S31508000960FF5001F0E1F8384601F09EF810F4604FA8
S3150800097003D0810404D513246BE7010C336899E787
S315080009804204E0D4030401D50F2462E70121F5E708
S3150800099014010020A00100201801002044010020B5
S315080009A0040100202DE9F00FBB4FBC4B3A6879686B
S315080009B01C68BB4D03460E0E100E4FEA901AC0F384
S315080009C08309C2F30748C2F3072C360100F0030077
S315080009D0D2B283F800A083F80190987083F8038058
S315080009E083F804C05A71DE80B3F806B02D6883F820
S315080009F05640C1F30722C1F307401FFA8BF65FFA88
S31508000A0082FC46EA101B4FEADC1A00F00F00C2F31C
S31508000A108019C2F34018C2F30016A3F854500025F3
S31508000A20012CA3F806B086B0187283F809A083F8DB
S31508000A300A9083F80B801E735D7340F2ED80022CDA
S31508000A4000F0C880BE680CF03F04FF689549620054
S31508000A50CCF3801983F819909A7693F81A800C6863
S31508000A604A68380EC6F3C01C00F0030548EA0C0BAA
S31508000A704FEAD01AC0F34119AD0006F07F06C0F35D
S31508000A80820083F81AB0DE7683F81CA083F81D90DE
S31508000A909877DD7793F81FB0C7F3074C01250CEA62
S31508000AA00509C7F30728CDF804904BEA9C1BCCF33D
S31508000AB0401A83F81FB04FEAD81C83F820A0DDF847
S31508000AC004A0CDF808C0002083F82100C8F38019D7
S31508000AD083F822A0DDF808A0CDF80C9083F823A0AF
S31508000AE0C8F3401CDDF80CA0CDF810C083F824A08C
S31508000AF0C8F30019DDF810A0CDF8149083F825A0E6
S31508000B00C4F30746DDF814A0C8F38109C7F3460CF9
S31508000B103602270E08F0030883F826A083F82790E4
S31508000B2083F8288083F829C083F82A5083F82C7024
S31508000B30DE85DE8DC4F30727B6B23E432406DE857E
S31508000B401C631F6B160E47EA06441C631F6BC2F331
S31508000B50074647EA06241C638C681F6BC968C2F3FC
S31508000B60072CC4F307464CEA070C3606270ED2B202
S31508000B70C3F830C083F8342083F835709E639A6BC7
S31508000B80C4F3072642EA06429A639E6BE4B246EA33
S31508000B9004229A639E6B46EA11649C6393F83C6050
S31508000BA0C1F3074202F00F04240246EA121283F840
S31508000BB03C20DC87DA8FC1F3072492B22243C1F3C3
S31508000BC04601DA8783F8401083F8415006B0BDE83D
S31508000BD0F00F704701F03F010C041C61BE681A69EA
S31508000BE0300E42EA00251D611C69C6F3074141EA39
S31508000BF004021A611D6901200024451944F1000107
S31508000C00CA0442EA5534E8044FF40075C6F3072CC3
S31508000C10DC6498641D6516E702F00306B2021A61E1
S31508000C201C69BE68C9B244EA810018611D69C6F329
S31508000C300742340E02F0030045EA941B04F007014C
S31508000C40C4F3C20540005409C2F38202C3F810B0C7
S31508000C501D7559759C75DA7518761D7EC6F3072CB1
S31508000C6045EADC1119761C69187E1D7A0122811C59
S31508000C7002FA01F002FA05F204F1010AC517A0FB0F
S31508000C80020102FB0511A0FB0A450AFB01551A657C
S31508000C90C3E91245D7E600BF04010020140100206D
S31508000CA0440100201801002038B51A4B1968032999
S31508000CB0054617D0022918D8B0F5805F12D0B0F5CE
S31508000CC0006F15D00020FFF77BFB044658B9124A7F
S31508000CD010461475146054609460D460146100F072
S31508000CE093FE00E02724204638BD0024204638BD60
S31508000CF00120FFF765FB04460028F4D1064B184689
S31508000D001C751C605C609C60DD601C6100F07CFEEC
S31508000D10E9E700BF140100202C01002040F2A013CF
S31508000D20C2F2000310B54022072418609A601846DC
S31508000D3000214FF480625C60D9601A6100F094FE6D
S31508000D402046BDE81040FFF7C1BA00BFF0B585B030
S31508000D5000240C2001218DF8074000F0F3FD4FF424
S31508000D600060C4F2020008210C2200F079FD4FF45D
S31508000D700060C4F2020009210C2200F071FD4FF454
S31508000D800060C4F202000A210C2200F069FD4FF44B
S31508000D900060C4F202000B210C2200F061FD0C2158
S31508000DA04FF400600A46C4F2020000F059FD4FF401
S31508000DB040600C22C4F20200022100F051FD4FF4FB
S31508000DC000604FF4706301250227C4F2020002A9ED
S31508000DD002938DF80D508DF80C708DF80E408DF835
S31508000DE00F5000F08FFC4FF440600422C4F202005A
S31508000DF002A9029200F086FC4FF40060C4F20200D9
S31508000E0002A94FF4805602968DF80F4000F07AFC3E
S31508000E104FF40060064602A9C4F2020002968DF855
S31508000E200C708DF80F4000F06DFC3046294600F036
S31508000E30B3FD4FF48000294600F084FD00F0D6FD8E
S31508000E40FFF7F2FB8DF807009DF8070018B19DF82B
S31508000E50070005B0F0BDFFF7F7FC8DF807009DF811
S31508000E600730002BF3D1134A134C13751046136041
S31508000E7053609360D360136100F0C6FD2046FFF708
S31508000E8091FD8DF807009DF8071051B19DF80730C0
S31508000E90002BDCD14FF40060FFF706FF8DF8070042
S31508000EA0D5E7B4F854000004FFF738FF8DF80700BB
S31508000EB0ECE700BF2C010020480100202DE9F8438B
S31508000EC0714D724E00214FF430542970C4F201045A
S31508000ED06F4D31602960E1626E4C6F4D21680229C1
S31508000EE018BFBDF82070914602BF4FEA52294FF449
S31508000EF0007749EAC35980461023402200264FF45A
S31508000F00806428462C612F606B60AA60EE604FF4FF
S31508000F10803400F0A9FD05E0802000F0FBFD38B91B
S31508000F20013C05D0802000F0F5FD013C0028F3D0F7
S31508000F301020FFF7CBF9064610B13046BDE8F88316
S31508000F4056494FF0FF329023084681E884008B60AB
S31508000F5002220123CA604B610E61112400F0B2FD22
S31508000F604FF480614C48EE604026AE602961C5F8B2
S31508000F7000906C6000F078FD2046FFF7A7F906465A
S31508000F800028DAD14FF430554446C4F201056A6B9D
S31508000F9040F22A6313404FF4004023BB00F0BAFD29
S31508000FA00028F4D000F0A6FD206000F0A3FD6060E4
S31508000FB000F0A0FDA06000F09DFDE06000F09AFD45
S31508000FC0206100F097FD606100F094FDA06100F0DB
S31508000FD091FDE0616A6B40F22A63134020344FF4B6
S31508000FE00040002BDAD0082000F094FD30B108202C
S31508000FF0042600F099FD3046BDE8F883022000F08B
S3150800100089FD20B1022000F08FFD022695E72020F9
S3150800101000F080FD20B1202000F086FD06268CE732
S315080010204FF4007000F076FD40BB4FF0FF3516E038
S31508001030E5B100F05FFD47F8040B4FF4001000F02F
S3150800104069FD98B100F056FD60604FF4001000F09D
S3150800105061FD58B100F04EFD0C347860033D4FF445
S315080010600010274600F056FD0028E1D140F2FF5057
S3150800107000F05AFD0A49002008605EE74FF4007048
S3150800108000F052FD072658E7E80000202801002056
S31508001090B401002014010020A0010020EC0000206B
S315080010A0000000202DE9F84F4FF43054C4F2010433
S315080010B0704D714E714F0021297031603960E162BF
S315080010C06F4C21686F4C022918BFBDF828909246CC
S315080010D002BF4FEA522A4FF400794AEAC35A8046B9
S315080010E010250023204640274FF480666560E3609C
S315080010F0C4F80090A760266100F0B6FC2846FFF702
S31508001100E5F8054610B12846BDE8F88F4FF0180BEC
S315080011102046E56084E8000CA760266100F0A4FC80
S315080011205846FFF7D3F805460028ECD156494FF044
S31508001130FF3281E804020123902208468A60CD60C6
S315080011400D614B6100F0BEFC4FF43057A946C4F25E
S315080011500107786B40F21A61014000293AD14FF431
S31508001160804000F0D7FC0028F3D0C9F5007BBBF11E
S315080011701F0F3AD85FEA9B0BEBD046460BF1FF33BD
S31508001180012456F8040B03EA040A00F0BBFC5C458C
S3150800119016D0BAF1000F06D056F8040B022400F058
S315080011A0B1FC5C450CD0B24602345AF8040B00F088
S315080011B0A9FC706800F0A6FC5C450AF10406F2D1A9
S315080011C0786B40F21A61014008EB840809EB840940
S315080011D00029C4D0082000F09DFC58B30820042537
S315080011E000F0A2FC2846BDE8F88FD8F8000000F009
S315080011F089FCD8F8040000F085FCD8F8080000F04F
S3150800120081FCD8F80C0000F07DFCD8F8100000F03E
S3150800121079FCD8F8140000F075FCD8F8180000F02E
S3150800122071FCD8F81C0000F06DFC08F1200809F1E3
S3150800123020098EE7022000F06DFC20B1022000F0A4
S3150800124073FC02255FE7102000F064FC20B1102033
S3150800125000F06AFC052556E74FF4007000F05AFCCA
S3150800126010B90A4A10604EE74FF4007000F05CFCB3
S31508001270072548E7E800002028010020B4010020DF
S3150800128014010020A0010020EC000020000000202E
S3150800129038B50446E0B1104A104B10680D25020413
S315080012A0402183E824001846996000224FF48061A3
S315080012B0DA60196100F0D8FB2846FFF707F80546FB
S315080012C008B1284638BD00F0EFFB2060284638BD37
S315080012D02625284638BD00BF44010020A00100206D
S315080012E000B583B000230193FFF78AF9012802D0DD
S315080012F0FF2003B000BD01A8FFF7CAFF0028F7D1F9
S315080013000198C0F34320F4E708B5FFF7E9FF04287E
S3150800131004D0FF2814BF0120022008BD002008BD04
S3150800132010B596B0FFF712FD044628B1074B012207
S315080013301A70032016B010BD04490A78684602F0F0
S31508001340FE030B70FFF72EFB2046F3E70400002090
S3150800135010B5084C0123237008B1207810BDFFF79B
S31508001360D3FF0028F9D1207800F0FE0121702078FB
S3150800137010BD00BF04000020F0B5ADF5037D10BB1D
S315080013805D1E03B34FF6FF74C0F27F04181901EB14
S315080013904024C1EB42274FF40076009602A8E219D2
S315080013A00023FFF78BFD70B9FFF7AEFF0128FBD0CE
S315080013B0204602A94FF4007208F0A0FFA4F50074B5
S315080013C02DB1013DE9E701200DF5037DF0BD284665
S315080013D0FAE700BFF0B5ADF5037D20BB5D1E13B37C
S315080013E04FF6FF74C0F27F04181901EB4024C1EBD5
S315080013F042274FF400764FF40072214602A808F0FF
S315080014007DFF009602A8E2190023FFF74BFE08B1FC
S31508001410052808D1FFF778FF0128FBD0A4F500744A
S315080014202DB1013DE7E701200DF5037DF0BD284606
S31508001430FAE700BF10B5164B1B78DB0798B00446D1
S3150800144002D5032018B010BD032906D8DFE801F03D
S3150800145003020D0770B10020F4E70420F2E7002824
S31508001460F9D1202010602046ECE74FF40071118076
S315080014700020E7E702A80192FFF794FA149A159B51
S31508001480500A019A40EAC35111602046DAE700BFC4
S31508001490040000204FF46053C4F2020300221968C6
S315080014A041F0010018609A60186843F2100120F0B4
S315080014B0847020F48030C2F20041186059601968BF
S315080014C082B021F480201860DA60009201921A68CE
S315080014D042F480311960184603E00099B1F5A06F0F
S315080014E009D0036803F40032019200994B1C00935B
S315080014F0019A002AF1D04FF46050C4F20200036842
S3150800150013F400320DD001210191019801280CD065
S315080015104FF46D43CEF200034FF00061996002B0BC
S315080015207047019201980128F2D14FF46053C4F232
S3150800153002034FF4E042196CC4F2000241F08050F5
S315080015401864116841F4404010609A689A60996876
S3150800155041F400409860996845F20C4241F4A05065
S31508001560C0F2407298605A60196841F080721A6039
S31508001570184601684FF460538A01C4F20203F8D58D
S315080015804FF47052C4F2020240F205601060996886
S3150800159021F003029A60986840F0020199609A68FF
S315080015A002F00C000828FAD1B2E700BF4FF47053D6
S315080015B0C4F202031A69002A09DA40F2231148F62E
S315080015C0AB10C4F26751CCF6EF50596058607047BB
S315080015D04FF47053C4F202031A6942F000401861CE
S315080015E0704700BF4FF47053C4F20203D8607047C7
S315080015F04FF47053C4F20203DA68D0030AD4D868E9
S31508001600C10601D505207047D96811F0EF0F03D040
S315080016100620704701207047DB6813F0020F0CBFE5
S3150800162008200720704700BF00B583B008238DF84F
S315080016300730FFF7DDFF8DF807009DF80700012842
S31508001640F7D09DF8070003B000BD00BF70B505468A
S315080016500E46FFF7E9FF082800D070BD4FF4705416
S31508001660C4F20204236923F440702061216941F41D
S3150800167000722261236943F0010020612E60FFF7A2
S31508001680D3FF216921F00102226170BD70B50546BC
S3150800169000292ED0012932D0022914BF4FF44076F2
S315080016A04FF40076FFF7C0FF082827D14FF470548F
S315080016B0C4F20204236923F44070206121690E43B1
S315080016C02661226922F0F8032361206940F00201AD
S315080016D00D432561226942F480332361FFF7A4FF95
S315080016E0216921F002022261236923F0F8012161B0
S315080016F070BD0E46FFF798FF0828D7D070BD4FF487
S315080017008076F7E72DE9F00F0E6884B00022884648
S3150800171013464FF0010B00968A4607E0DDF8049061
S31508001720A14539D04B1CAA1C102B54D0009E0BFA8D
S3150800173003F5591C05EA060C0BFA01F42640AC45DC
S31508001740019602F10205E9D1032606FA02F90768AD
S315080017509AF804806FEA09094E463E400660076813
S31508001760CDF80C9008FA02F908F1FF3849EA07099A
S31508001770B8F1010FC0F8009031D9C368039F9AF8F1
S3150800178007C0DDF804903B40C360C3680CFA02F258
S315080017901A43A145C260C5D1032304689AF80420F8
S315080017A0AB40DB431C400460046802FA05FC013ABE
S315080017B04CEA0404012A046033D9C2689AF807403F
S315080017C01340C360C26804FA05F31343C3604B1C95
S315080017D0AA1C102BAAD104B0BDE8F00F7047D0F8A8
S315080017E00880039E9AF806709AF8059006EA080893
S315080017F0C0F80880D0F8088009FA02F949EA08080A
S31508001800C0F80880D0F8048028EA0C0CC0F804C098
S31508001810D0F8049007FA03F39FB247EA0903436036
S31508001820ABE786689AF805709AF806201E40866027
S31508001830846807FA05FC4CEA040686604768019E38
S3150800184027EA06074760446802FA01F292B2224381
S315080018504260B2E7036919420CBF002001207047B5
S31508001860CB08083301F0070130B4890050F823503B
S315080018700F2404FA01F425EA040440F8234050F83A
S31508001880234002FA01F2144340F8234030BC704763
S315080018904FF46053C4F2020310B49A6802F00C01C4
S315080018A0042922D0082926D04FF41052C0F2F40297
S315080018B002604FF46053C4F2020321499C68C4F3E2
S315080018C003140C5D22FA04F242609C68C4F3822475
S315080018D00C5D22FA04F484609B68C3F34233C95C46
S315080018E022FA01F2C26010BC70474FF4D852C0F217
S315080018F0B7020260DDE75C68596814F4800F5C681B
S3150800190001F03F0214BF4FF4D8534FF41053C4F3F9
S3150800191088114FF4605414BFC0F2B703C0F2F40341
S31508001920C4F20204B3FBF2F303FB01F26168C1F3EC
S3150800193001435C1C6100B2FBF1F20260B9E700BF2B
S31508001940080000204FF46053C4F202031A6B19B959
S3150800195022EA00001863704710431863704700BFF7
S315080019604FF46053C4F202035A6B19B922EA000015
S315080019705863704710435863704700BF4FF460536D
S31508001980C4F202031A6C19B922EA000018647047F7
S3150800199010431864704700BF4FF46053C4F2020343
S315080019A05A6C19B922EA0000586470471043586403
S315080019B0704700BF4FF46053C4F202031A6919B99D
S315080019C022EA00001861704710431861704700BF8B
S315080019D04FF46053C4F202035A6A19B922EA0000A6
S315080019E05862704710435862704700BF08B5012116
S315080019F04FF40060FFF7ECFF4FF400600021BDE8EC
S31508001A000840FFF7E5BF00BFF0B44FF43053D0F8F5
S31508001A1004C08268C76806680469017DC4F20103C8
S31508001A204CEA02025D683A43324325F4FD402243FC
S31508001A3020F07F0002430A435A60F0BC704700BF9B
S31508001A4048F2A003C4F22523186070474FF43053B8
S31508001A50C4F20103186070474FF43053C4F201030F
S31508001A60186800F0030070474FF430530268C4F258
S31508001A70010330B49A6085684268C468D968006909
S31508001A802A4321F4FF61224321F0070102430A4356
S31508001A90DA6030BC704700BF4FF43053C4F201031C
S31508001AA01869C0B2704700BF42F6144382B0C4F248
S31508001AB00103C0180022019201900199086802B03A
S31508001AC0704700BF4FF430530268C4F2010330B4C4
S31508001AD05A6241689962C56882680469D96A406928
S31508001AE02A43224321F0F70102430A43DA6230BC53
S31508001AF0704700BF4FF43053C4F20103D3F8800097
S31508001B00704700BF4FF43053C4F20103C3F8800096
S31508001B10704700BF4FF43053C4F20103596B0842B3
S31508001B200CBF0020012070474FF43053C4F2010364
S31508001B3098637047DC23C4F227231860704700BFF8
S31508001B40028ACB8822F440521204F0B5120C0446DD
S31508001B501A4348890F898E880D4689892282A38966
S31508001B6023F4B05222F00C033E431A040643B3B2E0
S31508001B70100C43EA0006A681A28A22F440700304E8
S31508001B801E0C0E4385B0A6826846FFF781FE4FF409
S31508001B908051C4F201018C422CD04FF4A052C4F2F9
S31508001BA00102944226D0A089029B06B2002E26DBAB
S31508001BB02D6803EB830101EB8102AB00B2FBF3F165
S31508001BC048F21F53A089C5F2EB13A3FB015672090D
S31508001BD000B264251601002802FB151118DB0D0159
S31508001BE03235A3FB0553C3F34312324391B2218125
S31508001BF005B0F0BDA089039B06B2002ED8DA286886
S31508001C0003EB830606EB86054200B5FBF2F1D7E740
S31508001C10C8003230A3FB0013C3F342123243E5E790
S31508001C20838929B923F400510A04130C8381704768
S31508001C3099B241F400528281704700BFC905CA0DA6
S31508001C40828070478088C105C80D7047038819428D
S31508001C500CBF00200120704708B501214FF0007025
S31508001C60FFF7A8FE4FF000700021BDE80840FFF717
S31508001C70A1BE00BF40210164202141648021416644
S31508001C804FF0806100234FF00072C0F880104FF0CB
S31508001C908071036043608360C3600361436183614D
S31508001CA0C361036243628362C362036343638363FC
S31508001CB0C3638364C364036543658365C365036659
S31508001CC08366C366036743678367C367C0F8842070
S31508001CD0C0F888104FF40011C0F88C10C0F8A42082
S31508001CE04FF480714FF40032C0F89030C0F8943049
S31508001CF0C0F89830C0F89C30C0F8A030C0F8A830BA
S31508001D00C0F8AC20C0F8B010C0F8B430C0F8B8308D
S31508001D10704700BF4FF40042C4F2020202F5805336
S31508001D20116841F008001060996941F480109861C3
S31508001D30116841F0040010609A6942F400519961F3
S31508001D40986940F002029A61704700BF82B04FF46A
S31508001D500043C4F20203002201921A69890102F0C3
S31508001D601C02C00642EA104001F4F862104340F033
S31508001D7001014FF6FE7019611A46C0F2040002E02E
S31508001D800199814205D8019B591C01911369DB070A
S31508001D90F6D401984FF6FF72C0F20402904207D0BB
S31508001DA04FF40043C4F20203596988B202B070477F
S31508001DB00020FBE710B44FF4004383B0C4F20203DB
S31508001DC0002401941C695A6104F01C04C0068901A8
S31508001DD044F0030444EA104401F4F86004434FF65F
S31508001DE0FE711A461C61C0F2040102E0019888429D
S31508001DF005D8019B581C01901369D807F6D4019998
S31508001E004FF6FF72C0F20402881A18BF012003B009
S31508001E1010BC70472DE9F0414FF4004386B000220C
S31508001E20C4F2020300928046019202A81D690C467C
S31508001E30FFF72EFD03994FF45340CFF6CE604EF2CE
S31508001E40BF120B18C0F2E402934225F01C0500F2FB
S31508001E50358145F008054FF40043C4F202032046D5
S31508001E601D6100214FF40042FFF7A4FF002800F08F
S31508001E7021814FF080600090009A2AB100994B1E8C
S31508001E80009300980028F9D1D8F80010002900F02E
S31508001E9031814FF6FE75C0F20405019B01215A1CDB
S31508001EA020460192FFF752FF00F0040081B211B9F3
S31508001EB0019BAB42F1D9019A4FF6FF70C0F20400BC
S31508001EC0824200F0F7800023204619464FF48052DC
S31508001ED00193FFF76FFF002800F0EC804FF6FE75C0
S31508001EE0C0F20405019920464A1C01210192FFF718
S31508001EF02DFF00F0200083B213B90199A942F1D948
S31508001F00019A4FF6FF70C0F20400824200F0D280B8
S31508001F102046102100240194FFF718FF00F004065C
S31508001F20B5B2002D00F007814FF40067C8F820709D
S31508001F3000F0020399B2002900F0F7800020C8F8E3
S31508001F401400074608F1180393E80700D8F8046058
S31508001F50D8F80830D8F80C50D8F810401E43354346
S31508001F602C432043D8F82430D8F82860D8F82C40D9
S31508001F7001430A434FF4004CC4F2020C1A43D8F842
S31508001F803000DCF80050D8F834303243224348F2A7
S31508001F900F110243CFF6207129401A430A433A43E8
S31508001FA0CCF8002008F148010FC9D8F83860D8F8ED
S31508001FB03C70D8F84050D8F84440374347EA0506FD
S31508001FC046EA0405284340EA010422431343CCF8B1
S31508001FD00430D8F85810CCF80810D8F85C70CCF84B
S31508001FE00C70D8F86850D8F86440D8F86C00D8F85F
S31508001FF07030DCF81860D8F87410D8F8602045EA14
S31508002000040747EA00051D434FF6417445EA0100F7
S31508002010344040EA040343EA0246CCF81860D8F88C
S315080020207C10D8F8782041EA0207CCF81C70D8F85A
S315080020308030D8F88470D8F88850D8F88C4008F1E1
S31508002040900007C847EA030646EA050343EA04057B
S315080020504FF4104E45EA0004C4F2020ED8F89C303C
S31508002060DEF8180021430A4343F62375D8F8A01072
S3150800207042EA0304CFF6DE050C43054044EA0500B0
S31508002080CEF81800D8F8A450D8F8A830D8F8AC403C
S31508002090D8F8B000D8F8B810D8F8B4202B4343F4D1
S315080020A00003234303430B4343EA8200CEF80000B0
S315080020B0012000E0002006B0BDE8F0814FF2401094
S315080020C0CFF6E95047F63F020B18C0F27D1293424D
S315080020D002D845F00C05BEE64FF4F240CFF66C4048
S315080020E04FF4B4420918C0F26222914288BF45F003
S315080020F00405B0E6D8F82020D8F81430D00840EA0D
S31508002100530292B22046FFF755FE0028D2D06FF050
S315080021107F440094009E2EB1009F7D1E0095009975
S315080021200029F9D1D8F814700CE74FF48042C8F8A2
S315080021301420174606E7C8F82050F9E64FF410436E
S31508002140C4F202031A6842F001001860704700BF23
S315080021504FF41043C4F20203186800F001007047F8
S315080021602DE9F0430121B3B04FF0F050FFF7EAFB39
S3150800217047200121FFF7E6FB01214FF48040FFF7D6
S315080021800BFC0120FFF7D6FC00208E23064602250D
S31508002190C4F2020001A901938DF80A608DF808506F
S315080021A08DF80B608DF80950FFF7ACFA304601211F
S315080021B00B22C4F20200FFF753FB30460B22C4F28F
S315080021C002002946FFF74CFB304603210B22C4F2D6
S315080021D00200FFF745FB30460B220721C4F2020036
S315080021E0FFF73EFB4FF4C0504FF40062C4F2020002
S315080021F001A901928DF80A608DF808508DF80B60D8
S315080022008DF80950FFF77EFA0B214FF4C0500A46A5
S31508002210C4F20200FFF724FB4FF40060C4F2020088
S3150800222001A9322701978DF80A608DF808508DF8B4
S315080022300B608DF80950FFF765FA4FF4006001212D
S31508002240C4F202000B22FFF70BFB4FF400600421D7
S31508002250C4F202000B22FFF703FB4FF400600B22C7
S31508002260C4F202000521FFF7FBFA4FF4C0504FF401
S31508002270C043C4F2020001A901938DF80A608DF8E3
S3150800228008508DF80B608DF80950FFF73BFA4FF4AC
S31508002290C050C4F202000D210B22FFF7E1FA4FF4F9
S315080022A0C050C4F202000E210B22FFF7D9FAFFF73D
S315080022B0D3FCFFF743FFFFF74BFF0128FBD003A82A
S315080022C0FFF7D8FC002641F219684CF2F1094FF4E1
S315080022D000704FF0004120254FF400624FF480470C
S315080022E003960A960D900E961191149516961796C2
S315080022F018960B920897C0F22208C0F2070913E055
S315080023004C4523D0BDB22846FFF720FD032160F3D4
S315080023101F442846FFF71AFD60F30F04444515D0FD
S315080023204C4513D0202E3DD0B5B202212846FFF7E2
S315080023300DFD032160F31F442846FFF707FD60F3F0
S315080023400F04771C022144450E44D9D103A8294617
S31508002350FFF760FD20B9144840F2471102F094FFD8
S315080023604FF41040114A124C124B9460C4F202000A
S31508002370002111605160D2600261402259605A7191
S315080023809A8819604FF4C86161F30C020A499A8069
S3150800239080229960DB60DA70C360FFF7BBFC33B05C
S315080023A0BDE8F0833546D1E7F8A300080009002008
S315080023B080090020000200208002002042F6706397
S315080023C0C2F200030822002027211A70587099705B
S315080023D069225B204521DA7018715971704700BF70
S315080023E038B50E4CE37803F08000C1B211B1002570
S315080023F0284638BD65880A490A48AA04950C2A461B
S3150800240007F07CFFE0784FF41043C4F2020340F073
S3150800241080010122E17028469A6038BD000200203A
S315080024208002002014280020F8B5104CE57805F045
S315080024308000C5B2C5B90E4E0E4F0F493A883046D0
S3150800244007F05CFF3B88656019054FF41042080DDC
S31508002450C4F20202A0801023B02101202560A660E4
S31508002460A370E1705060F8BDFEE700BF00090020C8
S31508002470800900200828002014280020D0F8E83514
S3150800248010B5044618698047032184F81211002004
S3150800249010BD00BF08B590F81221D0F8E83580F8CD
S315080024A01321042180F81211D8688047002008BD3E
S315080024B008B5D0F8E435D96901B18847002008BDC8
S315080024C008B5D0F8E435196A8847002008BD00BF6A
S315080024D008B5D0F8E435596A8847002008BD00BF1A
S315080024E0D0F8E83510B5044658698047012184F8C4
S315080024F01511002010BD00BFD0F8E83510B5044608
S3150800250098698047D4F8E41520464A680021904720
S31508002510002084F8150110BD002110B50B460446AD
S31508002520402201F013F9802140220023204601F0C1
S315080025300DF9D4F8E835A078012284F812215968F3
S315080025408847002010BD00BF10B582B06946044612
S3150800255000F030F99DF8001001F01F03012B0FD091
S3150800256009D3022B11D0204601F0800101F068F949
S31508002570002002B010BD2046694600F0D1F9F7E701
S315080025802046694600F0B2F9F2E72046694600F0AF
S3150800259041F9EDE770B5044649B990F81131022BB7
S315080025A019D094F8161101290CD0002070BDD0F866
S315080025B0E4355B69002BF8D090F81221032AF4D190
S315080025C09847F2E721482369026800215A600020EB
S315080025D084F8161170BDD0F83821D0F824319A4203
S315080025E011D9C078D4F828110128C3EB020208BF14
S315080025F0C918C4F8382108BFC4F82811204692B271
S3150800260000F0A4F8CDE7D0F83C51B5FBF3F603FB90
S3150800261016565EB9AB4209D8D0F84021954205D284
S31508002620324600F093F8C4F84061BAE7D4F8E405F6
S31508002630C16819B194F81231032B03D0204600F073
S31508002640A9F8AEE720468847F8E700BFC00F002084
S3150800265010B5044629B990F8111103290CD00020A9
S3150800266010BDD0F8E4359B69002BF8D090F81221FC
S31508002670032AF4D19847F2E7D0F89023D0F87C33B0
S315080026809A4214D9C078D4F880130128C3EB020201
S3150800269008BFC918C4F8902308BFC4F880139A4223
S315080026A028BF1A46204692B200F05AF8D7E7D0F863
S315080026B0E4150B691BB190F81221032A03D02046B2
S315080026C000F058F8CBE79847F9E700BF2DE9F04145
S315080026D0069D044616461F46884601F0B9FC204664
S315080026E04146C4F8E475C4F8E855C4F8EC6500F04A
S315080026F0DDFFD4F8E835186880472046BDE8F04184
S3150800270001F0FEBCD0F8E43510B504461A689047C7
S31508002710D4F8E80581688847002010BD08B5D0F8C8
S31508002720E4355A689047002008BD00BF13460A469C
S31508002730022110B5C0F83C31C0F8383180F81111C3
S315080027400021044601F05EF8002010BD10B50C46C5
S3150800275013460021224601F055F8002010BD00BF9F
S3150800276010B50C4613460021224601F02BF800202E
S3150800277010BD00BF38B50021042504460A460B469D
S3150800278080F8115101F03EF8204600F071FF002054
S3150800279038BD00BF38B50021052504460A460B4654
S315080027A080F8115101F00EF8204600F061FF002074
S315080027B038BD00BF90F8CC350B7090F8CD254A701F
S315080027C090F8CE3590F8CF2503EB02224A8090F890
S315080027D0D03590F8D12503EB02228A8090F8D235BD
S315080027E090F8D32503EB022293B2CB800121C0F8DF
S315080027F0403180F81111704710B58021044601F068
S315080028001FF82046002101F01BF82046BDE81040BD
S3150800281000F02EBF70B54B788A88012B0C4605460A
S31508002820D6B21CD003D3032B25D0002070BD90F858
S315080028301231022B17D0032B23D1130646D406EBED
S31508002840860600EBC60696F87603002848D1264A7F
S315080028501060284624490222FFF768FFE5E790F84A
S315080028601231022B11D1002EDFD0802EDDD0314659
S3150800287000F0E6FFD9E790F81221022AF3D0032ADE
S3150800288019D0FFF7B9FF002070BD032BF9D14A888C
S31508002890002ACAD156B1802E08D0314600F0F0FF82
S315080028A0D5F8E41528468B68214698472846FFF749
S315080028B061FF002070BD49880029F1D1002EEFD0B4
S315080028C0802EEDD0314600F0BBFFE9E702F07F022B
S315080028D002EB820100EBC10393F81E010028B6D073
S315080028E0014901200860B4E7C810002038B590F8FF
S315080028F01231032B04460D4603D0FFF77DFF002057
S3150800290038BD0A79012AF8D8D0F8E4359A6890478C
S31508002910E8880028F3D12046FFF72CFFEFE700BF31
S3150800292070B54B7882B00C460546092B11D8DFE8FE
S3150800293003F0374A105F107492100517E288012ACF
S3150800294007D190F81211022900F02C81032900F012
S31508002950D28028462146FFF74FFF002002B070BDFF
S31508002960A178A54E01293170F3D890F812010228F2
S3150800297000F01C810328ECD1002900F0318195F87C
S315080029801011012908D02846FFF7C8FE31782846D5
S3150800299085F81011FFF7B6FE2846FFF7EBFEDCE7D1
S315080029A090F81211881E0128D3D8944BD5F818210F
S315080029B0012119600AB10320186028468F490222AE
S315080029C0FFF7B4FEC9E790F81201831E012BC0D8A1
S315080029D061880129C1D1D5F8E40500228368C5F8C4
S315080029E018212846214698472846FFF7C3FEB4E72C
S315080029F06388012B00F0EE80022BAED1A18811F07E
S31508002A00FF0FAAD10269080A431E5268042B7AD816
S31508002A10DFE803F0828A868E7600A188002998D19D
S31508002A20E088002895D1668895F8122106F07F037C
S31508002A30032A1E468DD0284685F81431194600F01B
S31508002A403FFF2846FFF796FE002E00F0BF800220C3
S31508002A5085F8120181E76088020A531E062B3FF6A5
S31508002A6078AF01A151F823F0D52A0008972A000863
S31508002A70852A000853290008532900085329000805
S31508002A8053290008C1B205293FF663AFDFE801F014
S31508002A9081786F665D54D5F8E435A8789A6A0DF1A1
S31508002AA006019047014602204870C5F8F015BDF8A2
S31508002AB00630002B3FF451AFE288002A3FF44DAFB1
S31508002AC0934228BF134628461A46ADF80630FFF744
S31508002AD02DFE42E7D5F8EC15A8780B680DF106012E
S31508002AE09847E288402A014603D095F81201012842
S31508002AF0DDD10823E1E700F58871FFF717FE2CE71B
S31508002B00052161F3061201233D4985F81631284649
S31508002B100A60FFF72FFE20E7012060F30612F2E7AE
S31508002B20032363F30612EEE7022161F30612EAE7CE
S31508002B30042060F30612E6E7D5F8EC25A878936931
S31508002B400DF1060198470146B1E7D5F8EC15A878C6
S31508002B504A690DF1060190470146A8E7D5F8EC3514
S31508002B60A8781A690DF10601904701469FE7D5F83E
S31508002B70EC15A878CB680DF106019847014696E74B
S31508002B80D5F8EC25A87893680DF106019847014613
S31508002B908DE7D5F8EC15A8784A680DF10601904737
S31508002BA0014684E71749FFF7C1FDD6E600293FF439
S31508002BB0F3AE0121032385F8101185F81231284652
S31508002BC0FFF7A0FD2846FFF7D5FDC6E6012185F8E3
S31508002BD01211C2E6D0F8E425C0F81831936800E768
S31508002BE0022285F8122185F810112846FFF796FD6E
S31508002BF02846FFF7BFFDB0E6CC100020C410002021
S31508002C00C00F0020D010002030B4F0B10378F3B123
S31508002C100446002314F8015F0133DBB2002DF9D115
S31508002C205C00A31CDCB2138003220C704A70027885
S31508002C305AB1022300255C1CE4B2CA540D5510F89B
S31508002C40012F0233DBB2002AF5D130BC70470224CB
S31508002C502346E8E730B5054683B0002303200193F1
S31508002C6001F050FAEB681A694FF454640192C0F205
S31508002C7003040FE001F046FAEB681A69019201991C
S31508002C80032000290CDB01F03DFAEB681969013CC9
S31508002C90019124D001990320002904F1FF34E9DACF
S31508002CA0019840F0010201920199196118694FF4DF
S31508002CB054620190C0F2030208E018690190019974
S31508002CC0C90709D51869013A019005D0019911F08B
S31508002CD0010F02F1FF32F0D1032001F013FA0020B0
S31508002CE003B030BD10B4C47814BB00EB82000333C4
S31508002CF09B10D0F8D0001BD051F8042B026001229B
S31508002D005C1E0431934204F0010411D034B151F829
S31508002D10044C022204319342046009D051F8044C51
S31508002D20046051F8044B0232043193420460F5D131
S31508002D30002010BC704700BF033270B49510D0F85D
S31508002D40D0401ED00B4620686A1E43F8040B02F0DA
S31508002D50010001220433954211D030B120680222C5
S31508002D6043F8040C0433954209D0266843F8046CEA
S31508002D70266843F8046B023204339542F5D101EB19
S31508002D808501084670BC70472DE9F00F0023012223
S31508002D904024012984B0C3708270848000F0BF800B
S31508002DA0002900F099800178427800914FF4006478
S31508002DB0C3600461002A00F0D4804FF460654FF4C4
S31508002DC088664FF480610395029601919B464FEA07
S31508002DD0421AAAF1200220230BF510650BF530667E
S31508002DE0C2F34014021D5345856146651ED04CB199
S31508002DF00BF512640BF53261402394615165043278
S31508002E00534513D0814603F1200705EB030806EB6B
S31508002E10030CE8194033F719C2F81880C2F854C0F1
S31508002E20D061976508325345EDD14846019C009913
S31508002E304461029CC0F8CC40002945D0009D0BF5A2
S31508002E40A06202EB4515AC1A0BF5A463203CC0F84A
S31508002E509020021DAB42C4F3401111D031B1C2F823
S31508002E6090300BF5A8630432AB4209D003F1200475
S31508002E70C2F890304033C2F894400832AB42F5D1DC
S31508002E80009C0BF5805202EB0435A91A0BF500538A
S31508002E90A1F58051C0F8D020021DAB42C1F3003124
S31508002EA012D031B1C2F8D03003F580530432AB42A8
S31508002EB00AD003F58054C2F8D03003F50053C2F89F
S31508002EC0D4400832AB42F4D10399C0F80C11002063
S31508002ED004B0BDE8F00F70470C254FF4A066002338
S31508002EE0C1720570C6804FF4606100954FF4806624
S31508002EF04FF4886506224FF40064C4F20403C4F252
S31508002F000401C4F20405C4F2040642700391029552
S31508002F100196C4F204049B46C360046157E708257A
S31508002F200226C1724FF4A0710570C18006724FF473
S31508002F30606100954FF480664FF4886504224FF46B
S31508002F4000644FF0A043C5F20001C5F20005C5F2C2
S31508002F5000064270039102950196C5F200049B464D
S31508002F60DAE74FF460634FF488614FF480640393A3
S31508002F7002910194934659E738B5037A0025012B47
S31508002F8004461ED0C168CA6842F04003CB60FFF70A
S31508002F9061FE607AE16800280CBF4FF450224FF4B6
S31508002FA0E8128A63142001F0BBF8E278012A06D1F8
S31508002FB0E068816821F03E0343F02A02826000201F
S31508002FC038BDC068617A836B65F3104309B143F471
S31508002FD080138363C2686FF386126FF396526FF39A
S31508002FE051426FF3D342C2602046FFF733FEE078C2
S31508002FF00128E4D1052161F34405E36845F020057D
S315080030009D60D2E7C3689A6842F001009860002084
S31508003010704700BFC3689A6822F0010098600020D4
S31508003020704700BF00B583B000230193019A42F0B0
S3150800303020030193019A61F38A1201920199C268E9
S31508003040116110694FF454630190C0F2030308E05C
S31508003050106901900199880609D51069013B01900C
S3150800306005D0019911F0200F03F1FF33F0D10320A9
S3150800307001F048F8002003B000BD00BF00B583B0DA
S3150800308000230193019941F010020192019BC06847
S31508003090036101694FF454630191C0F2030308E028
S315080030A001690191019AD10609D50169013B01918E
S315080030B005D0019A12F0100F03F1FF33F0D1032067
S315080030C001F020F8002003B000BD00BFC26808B5B3
S315080030D0D36801296FF35D736FF39E7308D009B93E
S315080030E043F080433220D36001F01AF8002008BD6F
S315080030F043F00053F6E700BFC368586900F00101C2
S3150800310081F00100704700BFC3685A69986910408A
S31508003110704700BF30B4C3684FF4006200216FF0F7
S315080031208044C8F200024FF0FF3599615C615D602A
S315080031305C619A61C27898698A4214BF0C46102469
S315080031400C2244F48724C4F23802224320EA0200FF
S3150800315010439861084630BC704700BFF8B505466D
S31508003160D0F80C012A6900210160166861F3CC26A3
S3150800317016600B46E97A012956D010212846FFF732
S3150800318051FF2846FFF77AFF2E6900224FF0FF33DA
S3150800319032617261B361F2616878002830D02946DD
S315080031A02C469646FF27A3691868C0F3076000F007
S315080031B08000C0B2002814BF4FF09040002018606D
S315080031C0C3F810E09F606B78013204349342EAD862
S315080031D0B3B100221746FF244B6D1868C0F3076089
S315080031E000F08000C0B2002814BF4FF090400020C5
S315080031F018601F619C606B78013204319342EBD8EA
S31508003200306940F480733361EA78012A07D102F500
S315080032108171C0F20101402060F3594131632846AB
S31508003220FFF778FF0020F8BD1668E868A027802415
S315080032304FF4001167F30F0346F00306166064F3B4
S315080032401F4364F30F014FF4907244628162C0F821
S31508003250043162F30F03C0F220034FF4A071C0F8E3
S31508003260083161F30F036FF31F43C0F80C3184E78D
S3150800327003699868C0F341014B1E022B02D8024A23
S31508003280D05C70470320704770A400080369826900
S3150800329098681168C0F34100022808D06FF30A0144
S315080032A011605A6842F48071596000207047032003
S315080032B060F30A01F4E700BF70B44B780022012BD3
S315080032C024D00B7800EB8304012505FA03F3646D1B
S315080032D063F31F422368C3F3072505F08005EDB2A3
S315080032E06DB98E68CD78C98866F30A0365F393438A
S315080032F061F3995343F0805343F400412160006918
S31508003300C3691A43C261002070BC70470C7800EB91
S31508003310840503FA04F363F30F02AC69DAE700BF26
S3150800332030B44A780023012A1C4613D00A7800EBE9
S315080033308201012505FA02F2496D62F31F4400690C
S315080033406FF3CF330B60C36923EA0404C46100201A
S3150800335030BC7047097800EB810502FA01F262F386
S315080033600F04A969EBE700BFF0B44B78012B3ED0F8
S315080033700A784D6900EB8204636D1C681A69EDB121
S315080033808F68EE19751EB5FBF7F5AE05B60D65F334
S31508003390DC4207FB06F666F312021A61C378012BB4
S315080033A016D0CB78012B1CD0097800EB810044F0AD
S315080033B00444436D1C600020F0BC70478D6865F3BB
S315080033C01202012565F3DC421A61C378012BE8D1A4
S315080033D00A780B6900EB8202526D5361CB78012B98
S315080033E0E2D14A79002A67D044F00054DCE70E7827
S315080033F04A6900EB8605AD692E682C69002A56D005
S315080034008B68CF7802EB030C0CF1FF3C62F31204D5
S31508003410BCFBF3F363F3DC44012F08BF67F35E7468
S315080034202C61C478012C51D0CB78012B47D052B1EE
S3150800343003690C785D6B012707FA04F42C435C6377
S31508003440CB78012B3BD00C7800EB840346F004467E
S315080034509C692660CC78012CADD1C578CB680978F3
S31508003460002DA8D192B200EB8100D11C8A10D0F8A9
S31508003470D000A0D053F8041B551E0433012A01605E
S3150800348005F00105214696D035B153F8044C0221C2
S3150800349004338A4204608ED053F8044C046053F80F
S315080034A0044B023104338A420460F5D183E762F3A0
S315080034B0120463F3DC44B3E744F0805474E7046908
S315080034C0A368DC0509D446F00056BCE70C780B69FE
S315080034D000EB8404A4696361B2E746F08056B2E75C
S315080034E0F0B44B78012B82B02DD00C784A6900EBEA
S315080034F084056B6D1D681E690096F2B18E689DF88D
S3150800350000409DF802204E6166F30604012666F324
S31508003510C4028DF800408DF80220009A1A61C3781B
S31508003520012B3FD0097800EB810045F00442436D3A
S315080035301A60002002B0F0BC70479DF800409DF864
S3150800354002208E68E0E782694C691668156900955D
S31508003550002C2ED08B689C423FD99DF800404B61C9
S3150800356063F306048DF800409DF80230012464F3E5
S31508003570C4038DF80230009B1361C378012B25D054
S3150800358046F004431360C278002AD2D14B69002B57
S31508003590CFD003690A78596B012000FA02F20A4370
S315080035A05A63C6E70A780B6900EB8202526D5361CB
S315080035B0B8E79DF800709DF8025064F3060763F3B8
S315080035C0C4058DF800708DF80250D4E70C780B69A5
S315080035D000EB8404A4696361D2E79DF8003064F3C4
S315080035E006038DF80030BFE74B780978012B00EB0E
S315080035F0810006D0436D1A6842F400111960002054
S31508003600704780690368C3F3076202F08001CAB293
S315080036100AB143F0804343F400110160002070476B
S315080036204B78012B0B78C97800EB83000CBF8269B5
S31508003630426D1368881E6FF35553012898BF43F0EF
S31508003640805313600020704703699A69D86910404F
S31508003650000C704700EB810102694B6D996850694F
S315080036600840704703699869D969084080B270476D
S3150800367082B00122002362F3C40300210091C02214
S315080036808DF8023018238DF803208DF80030416D2F
S31508003690009A0A61C378012B06D100F2CC50486122
S315080036A00A684FF080220A6002B0704770B5044677
S315080036B0FFF76AFB62780126002384F8126184F812
S315080036C014318AB31946402503EB830004EBC00284
S315080036D082F81C31A2F8223182F81D6182F81F1186
S315080036E0C2F82451C2F82811C2F8301160780133A3
S315080036F09842E9D8C0B100231946402503EB830256
S3150800370004EBC20080F87433A0F87A3380F8751396
S3150800371080F87713C0F87C53C0F88013C0F8881374
S31508003720627801339A42E9D82046FFF773FC2046AF
S31508003730FFF722FC00212046FFF7C8FC2046FFF7CA
S315080037400DFD2046BDE87040FFF75CBC38B501F0BA
S315080037507F0404EB8405090600EBC50511D405F5BD
S315080037605D7185F87443002405F55C754C708A60B4
S31508003770CB70022B01D100230B71FFF79DFD0020B2
S3150800378038BD05F58E7185F81C4101254D708A6096
S31508003790CB70CC80EDE700BF08B501F07F03CAB255
S315080037A003EB830100EBC10112F0800F14BF01F592
S315080037B08E7101F55D71D2090B704A70FFF7B0FD85
S315080037C0002008BD70B501F07F0404EB840500EB0A
S315080037D0C50505F55D71002685F87443CA604B6119
S315080037E08E614E70C378012B05F55C7508BF0A61BA
S315080037F01CB1FFF7B9FD002070BDFFF771FE002070
S3150800380070BD00BF70B501F07F0404EB840500EBC2
S31508003810C50505F58E710126CA600A61002285F87C
S315080038201C414E7005F58C758A614B611CB1FFF71A
S315080038309BFD002070BDFFF753FE002070BD00BF42
S31508003840CAB2130610B511D401EB810300EBC30409
S3150800385004F55D7301F07F01D209012419709C708B
S315080038605A701946FFF7C0FE002010BD01F07F010F
S3150800387001EB810400EBC40303F58E73ECE700BF8C
S31508003880CAB210B5140611D401EB810300EBC304C8
S3150800389004F55D7301F07F010024D20919709C704C
S315080038A05A701946FFF7BCFE204610BD01F07F018D
S315080038B001EB810400EBC40303F58E73ECE700BF4C
S315080038C003690022186861F30A1202431A607047F6
S315080038D003695A6842F002005860032000F020BCD1
S315080038E02DE9F04F85B00446FFF706FC10B905B080
S315080038F0BDE8F08F2046FFF707FC83460028F6D080
S31508003900C0F3074808F00800C0B2002840F0C48099
S3150800391008F004085FFA88F3002B56D15FFA8BF596
S3150800392005F00203DAB212B1E16802264E61CBF362
S31508003930076303F08002D1B2002940F05C81CBF323
S31508003940072606F00803D9B2002940F0228105F0BF
S315080039500802D3B2002B40F0128105F01005E9B237
S31508003960002940F0E58006F01003D9B2002940F09E
S31508003970968106F02006F6B2002E40F07881CBF349
S31508003980074505F01003DAB2002A40F0658105F014
S315080039902005EDB2002D40F05481CBF3076303F008
S315080039A04002D1B2002940F041810BF00403DAB29B
S315080039B0002A9CD0E3685D6805F00401C8B20028B7
S315080039C040F016825D60012091E72046FFF74AFE27
S315080039D0074600285ED026464FF00009CDF804B009
S315080039E0A24626E003F00801CCB214B1B069082358
S315080039F0836003F01002D5B215B1B16910238B604C
S31508003A0003F04004E0B210B1B2694023936003F0BA
S31508003A100205E9B211B1B4690223A36003F080007C
S31508003A20C2B2002A40F0908104367F0809F10109E4
S31508003A302DD0F807F8D5DAF810205FFA89F8146956
S31508003A40506B0AEB880120FA08F58869EB01816852
S31508003A50DDB225430D40EBB2D907C3D540F21804B1
S31508003A60C2F20004536B2168012404FA09F023EA20
S31508003A7000035363B5694A68AC60504641469047AF
S31508003A809AF80350A54200F09A812346AAE7DDF882
S31508003A9004B05446012041E72046FFF7D5FD054608
S31508003AA0002843D0A2462646002705E001370436FB
S31508003AB06D080AF1280A39D0EA07F7D55FFA87F9B7
S31508003AC020464946FFF7C6FDC0B2C30716D5736D33
S31508003AD001219960E2788A4200F0818140F218005B
S31508003AE0C2F200004946036820461A68904794F8CF
S31508003AF00390B9F1010F00F06B81012000F0020379
S31508003B00DAB212B1716D0220886000F00803DAB2E9
S31508003B10002ACBD040F21801C2F2000120460B68F9
S31508003B209A689047716D08208860BFE70120EFE624
S31508003B30E3689F6927F010029A611D6A05F00F0075
S31508003B4000EB8001C5F3434204EBC107022A07F5DF
S31508003B505D7700F0DB80062A0BD104F2CC512046B3
S31508003B600822FFF7E9F8B869E368C5F30A154119A9
S31508003B70B961986940F010029A610120F3E6A248FB
S31508003B8001682046CA689047E36808205861012002
S31508003B90E3E69D4894F81221036800215B698DF8D5
S31508003BA00F1020468DF80F2098472269E068916823
S31508003BB04FF400634361A27ADAB1CB0719D594F8BA
S31508003BC01501012815D19DF80F10032911D1D4F834
S31508003BD00C311A6842F00100186019684FF46D42FA
S31508003BE0CEF2000241F003001860136943F00601A3
S31508003BF011610120ABE6A07A40B1D4F80C61D4F883
S31508003C000C316FF341066FF300061E6020697E4A89
S31508003C104168166821F001034360B1692046884768
S31508003C20E0684FF000424261012088E67648036862
S31508003C3020465A6A9047E1684FF080404861012063
S31508003C40B3E671490B6820461A6A9047E0684FF454
S31508003C50001141610120A0E66B4801682046CB6946
S31508003C609847E0684FF48012426101208FE62046AB
S31508003C70FFF70CFBE5682046ED68FFF7F9FA03281D
S31508003C8059D0012040220521A070A28061F38D251C
S31508003C90E168CD604FF4005501204D616FE6256956
S31508003CA06868002720F001026A6020463946FFF757
S31508003CB0B9F963785BB123463A46FF2599698D6061
S31508003CC0586D85606178013204338A42F6D301253E
S31508003CD0236965F30F070B204FF0FF3165F31F4784
S31508003CE09961DF61586118611A686FF30A121A60E0
S31508003CF02046FFF7BDFC4448E36802684FF480514C
S31508003D005961204613699847284632E647F6F07205
S31508003D102A40002A3FF42DAFC5F30A152A46F9684A
S31508003D202046FFF709F8F868BA69E3684119551992
S31508003D30F960BD611DE700234FF400700922A370E6
S31508003D40A08062F38D25A3E709EB89050AEBC50177
S31508003D5001F58E75B1696A69A869AC68D1F818C0A9
S31508003D60131AA34234BF9B46A3460BF1030E1FFA50
S31508003D708CFCBCEB9E0F1FD982421DD9E2B1E968C3
S31508003D8004E06C699C4216D9E31AAC689C4228BFC9
S31508003D901C46A3B242465046FEF7A4FFE968AB6943
S31508003DA00919E318E960AB61B0698269033492B214
S31508003DB0B2EB940FE5D8014680258D6034E6B9F15B
S31508003DC0000F03D19AF81131042B1FD02B4609E6B0
S31508003DD01FB994F81111052911D048468EE61869BD
S31508003DE0DAF87C33C0F312015A1ACAF88C2375E63E
S31508003DF0054B1A682046916A8847E368E2E520463B
S31508003E00FFF736FCE9E700BF180000205046FFF729
S31508003E102FFCDBE7704700BF704700BF704700BF45
S31508003E200020012108B5C4F20200FDF713FD10F1C8
S31508003E30FF3018BF012008BD00B5C7B0002168468D
S31508003E404FF48C7206F07EFA0848694604F016FEAE
S31508003E5048B9009828B19DF8080080F01001C1F310
S31508003E60001047B000BD0020FBE700BF74A400089F
S31508003E704AF27440C0F60000704700BF10B5074C00
S31508003E800749002320460A2284F8283204F04CFA0F
S31508003E9010B9012084F8280210BD00BFD4100020F4
S31508003EA094A4000810B50F4890F82832012B16D0B4
S31508003EB000F0BCFE00F1640403E000F0B7FE8442A3
S31508003EC008D34FF4A0504021C4F20100FDF7BEFE0E
S31508003ED00028F2D00448BDE8104004F0FFBD04F005
S31508003EE007FDE5E7D410002074A40008034890F8FD
S31508003EF02832012B00D0704704F0FABCD4100020F9
S31508003F0038B5144D95F82832012B044615D021787A
S31508003F1091B14FF4A050C4F20100FDF78FFE4FF4A3
S31508003F20A050C4F201008021FDF790FE0028F6D0CB
S31508003F3014F8011F0029ECD138BD294604F058FEB3
S31508003F400028E4DA0021284685F8281204F0D0FC77
S31508003F50DDE700BFD410002000B583B0FDF79AFA5C
S31508003F6001200146FDF7EEFC002001240225064645
S31508003F706946C4F2020000948DF804608DF8076063
S31508003F808DF80550FDF7BEFB20202146FDF704FD00
S31508003F9004202146FDF7D6FC4FF40060C4F2020067
S31508003FA006210822FDF75CFC4FF400600822C4F2E3
S31508003FB002000721FDF754FC4FF400604023C4F2C9
S31508003FC00200694600938DF806608DF807408DF863
S31508003FD004508DF80550FDF795FB4FF400608022DC
S31508003FE0C4F20200694600928DF80450FDF78AFB78
S31508003FF028462146FDF7A6FC4FF48060C4F202006D
S3150800400005210922FDF72CFC4FF480600922C4F231
S3150800401002000621FDF724FC4FF480606023C4F2F9
S315080040200200694600938DF804508DF805508DF806
S3150800403006608DF80740FDF765FB4FF0C060214626
S31508004040FDF79CFC01F05AF901F06AF9FCE700BF9C
S31508004050F0B50120002483B0C4F202040146FDF73E
S3150800406071FC00264FF4C8530327022269462046EE
S3150800407000938DF804208DF805708DF806608DF88C
S315080040800760FDF73FFB204608210A22FDF7E8FBFB
S3150800409020460B210A22FDF7E3FB0A2220460C21C3
S315080040A0FDF7DEFB01254FF40073204669460093B1
S315080040B08DF805708DF804608DF806508DF8076048
S315080040C0FDF720FB694620464FF4806200928DF882
S315080040D006508DF807508DF80570FDF713FB0A2179
S315080040E00A462046FDF7BCFB29464FF48040FDF7FB
S315080040F053FC80202946FDF733FC03B0F0BD00BF12
S31508004100704700BF10F1FF3008D31C2100BF4B1EBB
S3150800411000BF591EFAD110F1FF30F6D2704700BF22
S315080041204FF47A7303FB00F010F1FF3008D31C221A
S3150800413000BF511E00BF4A1EFAD110F1FF30F6D259
S31508004140704700BF202340F248000B80C2F20000EF
S31508004150704700BF08B590F81231032B01D0002034
S3150800416008BD00F0B1FF002008BD00BF08B500F08B
S31508004170ABFF002008BD00BF084608B501F01EF8D1
S31508004180002008BD10B581210446FFF705FB20462F
S315080041900121FFF701FB002010BD00BF10B58121EA
S315080041A0044640220223FFF7D1FA012140220223C6
S315080041B02046FFF7CBFA41F2003220460121C2F22F
S315080041C000024023FFF7FEFA002010BD10B50A785A
S315080041D012F0600F0B46044606D14A780A2A05D023
S315080041E00B2A14D0062A07D0002010BD0F49012239
S315080041F0FEF79CFA002010BD4888010A21290ED036
S315080042000B4917222046FEF791FA002010BD8B783D
S3150800421013B9064A1360E7E7FEF7EEFAE4E7DA8829
S315080042200449172A28BF1722ECE700BF40130020CD
S31508004230510000205A00002041F20030C2F200006E
S31508004240704700BF122340F2B4000B80C2F2000090
S31508004250704700BF042340F2B0000B80C2F2000092
S31508004260704700BF10B540F6C474C2F200044AF2A3
S31508004270A4400A46C0F600002146FEF7C5FC2046C3
S3150800428010BD00BF10B540F6C474C2F200044AF26D
S31508004290BC400A46C0F600002146FEF7B5FC20469B
S315080042A010BD00BF10B540F6C474C2F200044AF24D
S315080042B0C4400A46C0F600002146FEF7A5FC204683
S315080042C010BD00BF10B540F6C474C2F200044AF22D
S315080042D0D4400A46C0F600002146FEF795FC204663
S315080042E010BD00BF10B540F6C474C2F200044AF20D
S315080042F0E4400A46C0F600002146FEF785FC204643
S3150800430010BD00BF704700BF704700BF704700BFB1
S315080043100020FFF77FBD00BF0120FFF77BBD00BF70
S31508004320FFF77CBDFFF778BD72B6704762B6704777
S315080043304AF2F840C0F60000382100F0A5BF00BFD9
S315080043402DE9F04F594B83B000204FF4FA724AF228
S31508004350104840F2FF3B1C18861C6178185C45180B
S3150800436005FB022498FBF4FC04FB0CF4C4F5244476
S315080043700CF1FF35103403EB06091FFA85FA14B958
S31508004380DA4540F28F80985D99F80110451805FBCB
S31508004390022498FBF4F504FB05F4C4F52444103410
S315080043A01CB9013DACB25C457CD9B01C2428D2D1DD
S315080043B03F48EC2100F068FF4FF0FF354FF4D0443A
S315080043C0C4F2000400236361226842F400412160BC
S315080043D02068020404D501F059F823681804FAD4B1
S315080043E04FF4D044C4F20004226822F0020121608E
S315080043F0206840F0010323606268D30704D401F003
S3150800440045F86168CA07FAD5019C013F601E3B055D
S315080044104FF4D044C4F2000443EA00473D43E56143
S31508004420226822F0010121606068C10704D501F005
S315080044302DF86368DB07FAD44FF4C840C4F20000CD
S315080044400022D0F8001241F00103C0F80032D0F87B
S315080044501C1221F48043C0F81C32D0F80C1241F427
S315080044608043C0F80C32C0F8B022C0F8B422D0F8A5
S31508004470042222F48041C0F80412D0F8143223F43E
S315080044808042C0F81422D0F81C1241F48043C0F8C8
S315080044901C32D0F8002222F00101C0F8001203B045
S315080044A0BDE8F08F01900F4688E700BF20A60008F8
S315080044B094A5000838B54FF4D043C4F20003044667
S315080044C0986843010D463BD54FF4D043C4F2000328
S315080044D0D3F8802102F00101C3F88011D3F88001D6
S315080044E040F07C4242F40011C3F88011C3F88451AD
S315080044F0A278E57820786178120442EA05650543D2
S3150800450045EA0120C3F88801A279E579207961791D
S31508004510120442EA0562024342EA0120C3F88C010A
S31508004520D3F8801141F00102C3F880219868400150
S3150800453005D41C4600F0AAFFA3685901FAD538BD70
S3150800454002484FF4A07100F09FFEBDE794A500084D
S315080045504FF4D043C4F20003DA6812F0030110D016
S31508004560D3F8B01140F26762B2EB515F0BD000206E
S315080045704FF4D043C4F20003DA6842F02001D96050
S31508004580704708467047D3F8B8110170D3F8B821B8
S31508004590110A4170D3F8B821110C8170D3F8B821EB
S315080045A0110EC170D3F8BC210271D3F8BC110A0AE6
S315080045B04271D3F8BC110A0C8271D3F8BC31190EBA
S315080045C0C1710120D4E700BFFFF7AEBE10B500F0F9
S315080045D0F5FA00B910BDFFF723FC0028FAD000F061
S315080045E005FF00F00DFB00F0EBFA4EF60853CEF28D
S315080045F0000320F0604020F07F021A6000F0E0FA25
S315080046004468FFF793FEA04710BD00BFF8B5571ED4
S31508004610BFB20AB30E1A441C825DC343E719F918E0
S31508004620027001F0010500F031FFBC4215D035B12A
S31508004630A05D04F8010B00F029FFBC420ED0A25D74
S31508004640254605F8012B00F021FFAB5D63706C1C55
S3150800465000F01CFFBC42F2D1F8BDF8BDF8BD00BFA2
S3150800466010B5044600F012FF4BF6FF73C0F60003C0
S315080046709C4205D94FF6FF70C0F60000844279D9EE
S3150800468000F004FF4FF6FF71C0F600018C4205D911
S315080046904FF6FF72C0F60102944269D900F0F6FEA1
S315080046A04FF6FF73C0F601039C4205D94FF6FF701B
S315080046B0C0F6030084425FD900F0E8FE4FF6FF71AA
S315080046C0C0F603018C4205D94FF6FF72C0F6050203
S315080046D0944255D900F0DAFE4FF6FF73C0F605038B
S315080046E09C4205D94FF6FF70C0F60700844245D9AB
S315080046F000F0CCFE4FF6FF71C0F607018C4205D9D3
S315080047004FF6FF72C0F6090294423DD900F0BEFE8C
S315080047104FF6FF73C0F609039C4205D94FF6FF70A2
S31508004720C0F60B0084422DD900F0B0FE4FF6FF719B
S31508004730C0F60B018C4205D94FF6FF72C0F60D0282
S3150800474094420DD900F0A2FE4FF6FF73C0F60D0392
S315080047509C4203D90820B4F1016F02D3FF2010BD93
S3150800476007200A4A00EB400102EB8103187A10BDC4
S315080047700120F6E70020F4E70220F2E70420F0E73C
S315080047800320EEE70620ECE70520EAE774A6000812
S315080047902DE9F84306460068FFF762FFFF283AD07E
S315080047A0FCF704FFF320FCF71DFFFCF721FF0128A7
S315080047B037D0002418E054F808202C1D974224D13D
S315080047C0D6F800804F6805EB080900F05FFE4846FA
S315080047D03946FCF73BFF082817D155F808008742E9
S315080047E013D1B4F5007F1AD03319D6F800805F6864
S315080047F004EB080900F04AFE39464846FCF726FF4E
S31508004800251D082806EB0501D5D00024FCF7E0FE97
S315080048102046BDE8F88300242046BDE8F883012435
S31508004820F4E7FCF7D5FE0024F2E700BF124A9042EF
S3150800483038B504460D461CD04FF44043C0F6000375
S31508004840994208D0FFF7A4FF10B1E805C10D19B1C8
S315080048500024204638BD14462268954207D02046D3
S31508004860294640F8045B4FF40072FFF7CFFE204656
S3150800487038BD024CE9E700BF441300204815002064
S315080048802DE9F84F064600684FEA512A9946431C17
S315080048900C4615464FEA4A2A70D0824507D030465C
S315080048A05146FFF7C3FF0646002864D00068241A5D
S315080048B031190C1D371D00F0E9FD40F2FF18E31B06
S315080048C009F1FF3B43450BF0010B0AF5007A40D886
S315080048D015F8012BB9F1010904F8012B2DD0BBF10C
S315080048E0000F0BD000F0D2FDE01B40453AD815F872
S315080048F0011BB9F1010904F8011B1ED000F0C6FD21
S31508004900E31B434509F1FF391AD815F8012B04F8BA
S31508004910012B00F0BBFDE01B4045E8D93046514667
S31508004920FFF784FF0646071D28B33C4615F8011B0A
S31508004930B9F1010904F8011BE0D10120BDE8F88F9F
S3150800494030465146FFF772FF0646071D98B13C46AA
S31508004950DBE730465146FFF769FF064658B1071DA3
S315080049603C46B5E730465146FFF760FF064610B1AC
S31508004970071D3C46BBE70020BDE8F88F3046514688
S3150800498040F804AB4FF40072FFF740FE306884E746
S3150800499041F2485241F24433C2F20002C2F2000325
S315080049A04FF0FF3111601960704700BF70B50446BB
S315080049B00D461646FFF754FEFF2816D0601E40190E
S315080049C0FFF74EFEFF2810D04FF44043620AC0F6A8
S315080049D00003B3EB422F0CBF054806482146324672
S315080049E02B46BDE87040FFF74BBF002070BD00BFE7
S315080049F04413002048150020F8B505460E46FFF773
S31508004A002FFE0446681E8019FFF72AFEFF2C05466E
S31508004A104CD0FF284AD0844248D8022C46D90B28C5
S31508004A2044D8FCF7C3FDF320FCF7DCFDFCF7E0FDFA
S31508004A30012837D0204E2B1B03F0010700F026FD76
S31508004A40022136F81400FCF721FE08282AD1013481
S31508004A50E4B2A5422CD3D7B100F018FD022136F8EE
S31508004A601400FCF713FE08281CD1611CCCB2A54221
S31508004A700DD21DE000F00AFD36F814000221FCF7FD
S31508004A8005FE631C0828DCB20CD1A54210D300F041
S31508004A90FDFC022136F81400FCF7F8FD621C082814
S31508004AA0D4B2E7D0FCF794FD0020F8BD0020F8BD8D
S31508004AB0FCF78EFD0120F8BD44A60008F0B5104BA2
S31508004AC01A68013283B019D003F114009F685E6832
S31508004AD0DD681C6907C8BB195B191B19181841182A
S31508004AE08B1802AA584242F8040D4CF28810C0F6F8
S31508004AF000000421FFF75AFF03B0F0BD0120FBE7D1
S31508004B00441300204CF204004FF440414CF20803D1
S31508004B10C0F60000C0F60001C0F600034CF20C0215
S31508004B2070B4C0F600020D6804681E684CF21003E3
S31508004B30C0F600034CF214016019C0F600011568AE
S31508004B401C6809684CF218028019C0F600024CF27B
S31508004B5088134019C0F60003001912681B6841182B
S31508004B608A18D018D0F1010038BF002070BC7047F1
S31508004B700A4808B50368013302D0FFF709FE58B1A1
S31508004B80074801684B1C05D0FFF702FE003018BF26
S31508004B90012008BD012008BD08BD00BF4413002040
S31508004BA0481500204FF44040C0F60000704700BF8B
S31508004BB0FFF7EEBEFFF7FABEFFF71EBFFFF7A2BF6D
S31508004BC0FFF7F0BF08B5FFF779FF00B908BDBDE8E4
S31508004BD00840FFF7CDBF00BF4EF21003CEF2000328
S31508004BE041F24C7249F23F000021C0F20200C2F2C3
S31508004BF000021960586005209960186011607047B6
S31508004C004EF21003CEF2000300221A60704700BF6E
S31508004C104EF21003CEF200031868C30303D5024907
S31508004C200A68531C0B6070474C1700204EF210039D
S31508004C30CEF200030449186810F4803F086802D0D1
S31508004C4001300860704770474C17002038B5054694
S31508004C504FF4A0502021C4F20100FCF7F7FF012809
S31508004C60044602D00024204638BD4FF4A050C4F2B2
S31508004C700100FCF7E7FF2870204638BD10B54FF451
S31508004C80A05484B00023C4F20104694620464FF4B8
S31508004C906142ADF80430ADF80630ADF80830ADF82D
S31508004CA00C300C230092ADF80A30FCF749FF204679
S31508004CB00121FCF7B5FF04B010BD00BF4029F8B5C7
S31508004CC00E4607464AD84FF4A050C4F20100802188
S31508004CD0FCF7BCFF002830D123487A2100F0D4FA2B
S31508004CE056B3002407E0832101341F4800F0CCFAAC
S31508004CF0A3B29E421FD900F0C9FB4FF4A050C4F2DC
S31508004D00010080213D5DFCF7A1FF0028EBD04FF4A0
S31508004D10A050C4F201002946FCF790FF4FF4A050BA
S31508004D20C4F201008021FCF791FF0028F6D0013477
S31508004D30A3B29E42DFD8F8BDF8BD4FF4A050C4F226
S31508004D4001003146FCF77AFF4FF4A050C4F2010087
S31508004D508021FCF77BFF0028F6D0C1E702487621C0
S31508004D6000F092FAAFE700BFE0A600082DE9F0418F
S31508004D701F4C257880464DB91E4E3046FFF766FF14
S31508004D800128074627D00020BDE8F0811A4E194FA2
S31508004D903078411C7818FFF759FF012805460AD0D4
S31508004DA0FFF744FF154B1A6864329042EBD900208E
S31508004DB02070BDE8F08130783A78411CCBB29A422F
S31508004DC03370E0D14046791CFFF720FC00222270A0
S31508004DD02846BDE8F08130780028D4D0FFF726FFB2
S31508004DE00649054B08601D7027702846BDE8F08106
S31508004DF09817002054170020501700209C170020F1
S31508004E00012838B504460D4604D910484FF4CD712B
S31508004E1000F03AFA0E4A04EB440002EBC003197C90
S31508004E205C7C8C4210D0DC6825705A7CD96858683E
S31508004E30541C4A1C82425C74DA6003D91968012042
S31508004E40D96038BD012038BD002038BD6CA70008E0
S31508004E50A4170020012838B504460D4604D90F4882
S31508004E604FF4DE7100F010FA0D4A04EB440402EB2D
S31508004E70C403587C80B19968087828709A685C7C65
S31508004E805868511C013C81425C74996003D91A68C0
S31508004E9001209A6038BD012038BD00BF6CA7000804
S31508004EA0A41700202DE9F04F41F2D47585B0C2F25F
S31508004EB000050395039E41F2A47441F69807C2F2D1
S31508004EC000044FF0010EC2F200074FF0400A06EB4D
S31508004ED00E0C41F2A07807EB0A0640F2C803C2F2AC
S31508004EE00008C2F200036660039E0093002541F69F
S31508004EF0E00040F2940240F2680307EB0E0904F161
S31508004F00180BA574E56265743D70C8F8005084F8FE
S31508004F102950C2F200000CF13F057146C2F20002A8
S31508004F20C2F2000386F800E0C4F814B084F82AE058
S31508004F3084F810A0C4F80890C4F80C90C4F800903F
S31508004F4084F828A0C4F820C0C4F824C0C4F818C03F
S31508004F50E561FDF7BBFB05B0BDE8F08F08B541F686
S31508004F60E000C2F20000FEF7B3FC0020BDE80840EE
S31508004F70FEF750BF3F292DE9F0418846074654D829
S31508004F802D4E41463078FFF73BFF012803D02B48CA
S31508004F909E2100F079F9B8F1000F44D008F1FF33EB
S31508004FA003F0010500F072FA30783978FFF728FF28
S31508004FB0012803D02148A72100F066F901244445B9
S31508004FC031D27DB100F062FA3078395DFFF718FF0B
S31508004FD0A04203D01948A72100F056F90134A0B21F
S31508004FE0404527D200F052FA395D3078FFF708FFBE
S31508004FF0651C01284FF0A701104801D000F044F9BC
S3150800500000F044FA795D3078FFF7FAFE01284FF090
S31508005010A7010A4801D000F037F96C1CA1B2414536
S31508005020E0D3BDE8F081BDE8F08104489A2100F09C
S315080050302BF9A5E7BDE8F081981800206CA70008B1
S315080050402DE9F0411B4D80461B48FEF749FC2C789C
S3150800505054B91A4E1A4831460078FFF7FBFE012864
S315080050601ED00020BDE8F081164E154B3178134F3F
S3150800507018784A1CB918FFF7EDFE01280446F0D146
S3150800508030783A78411CCBB29A423370E9D140461F
S31508005090791CFFF7BBFA00222A702046BDE8F0818A
S315080050A031780029DDD0074B28701C702046BDE8F2
S315080050B0F08100BFD41E0020E018002058180020F8
S315080050C0D4170020DC1800202DE9F041364E34783C
S315080050D0012C82B004D935484FF4EE7100F0D4F8AB
S315080050E0334B04EB440003EBC004617C002958D021
S315080050F0402934BF88464FF0400830782D4F0DF1CF
S315080051000701FFF7A7FE08F1FF35012805F001059D
S3150800511004D026484FF4927100F0B6F89DF807209F
S315080051200124A0453A7036D995B130780DF10701BA
S31508005130FFF790FEA04204D01C484FF4927100F08D
S31508005140A3F89DF8070038550134E3B2984522D9EB
S315080051500DF107013078FFF77DFE651C01284FF435
S315080051609271124801D000F08FF89DF80710307838
S3150800517039550DF10701FFF76DFE01284FF49271BD
S315080051800A4801D000F080F86C1C9DF80700E2B2CE
S3150800519090457855DCD80848064A81214346FEF7EB
S315080051A031FB02B0BDE8F081981800206CA7000812
S315080051B0A417002018180020E01800202F4B00EB39
S315080051C0800003EBC0012DE9F041B1F88C73002F84
S315080051D049D02B4E7A1E347802F00105FFF72CF8D9
S315080051E001782046FFF70CFE012804D0254840F236
S315080051F0431100F049F80124A74234D98DB1357816
S31508005200FFF71AF8015D2846FFF7FAFDA04204D019
S315080052101C4840F2431100F037F80134A0B2874227
S3150800522021D996F80080FFF707F8015D4046FFF799
S31508005230E7FD651C012840F24311124801D000F031
S3150800524023F83478FEF7F8FF415D2046FFF7D8FDCE
S31508005250012840F243110B4801D000F015F86C1CE8
S31508005260A3B29F42DDD8FEF7E7FF024603480121B5
S315080052704023BDE8F041FEF7A5BA00BFE0180020BC
S31508005280D41700206CA7000808B500F0FFF8FCE763
S3150800529010B500F0F7F8012806D000F011FB18B198
S315080052A00B4C2378012B00D010BDFFF7BFFC094932
S315080052B00A6802F51C5310339842F5D30020207073
S315080052C000F008FB0028EFD1BDE81040FFF77EB9D3
S315080052D0D51E0020D81E002008B541F6D563C2F2B7
S315080052E0000301221A70FFF7A1FC41F6D861C2F249
S315080052F000010860BDE80840FFF7CABF08B5FFF718
S3150800530063F900F0C1F8FFF767FCFFF751FC00F0FE
S31508005310BFFA00F013F8BDE80840FFF7DDBF00BF8D
S3150800532008B500F0B3F8FFF773FC00F0E5FB00F0F2
S315080053301DF8BDE80840FFF7ABBF00BF10B540F247
S31508005340E404C2F2000400F0A3F8FEF7F9FF012313
S315080053502370FFF793FC00202070FFF7A3FD0221BE
S31508005360217004F0B9FE0322227010BD08B51D484D
S31508005370FFF7EEF80128034617D01A48FFF7F6FCA0
S3150800538001281CD01748FFF75BFE012822D01548D4
S3150800539004F00EFF012800D008BD134B1148032264
S315080053A01A70BDE8084000F093B80F4A0D4813700C
S315080053B000F08EF80B48FFF7D9FC0128E2D10A4B1A
S315080053C008480021197000F083F80648FFF738FEF0
S315080053D00128DCD10449034802220A7000F078F853
S315080053E0D5E700BFDC1E0020E4000020FFF7B6BDAD
S315080053F070B5134C2378012B06460D461BD03BB1DE
S31508005400022B0CD0032B11D0BDE8704000F058B821
S315080054103046E9B2FFF752FC2378022BF2D1304628
S31508005420E9B2FFF7A7FD2378032BEDD13046E9B2A1
S3150800543004F08EFEE8E7C9B2FFF73CF82378DEE70A
S31508005440E4000020054B1878411ECBB2012B01D988
S3150800545040207047024A32F813007047E4000020E3
S31508005460F8A70008054B1878411ECBB2012B01D9C5
S3150800547040207047024A32F813007047E4000020C3
S31508005480FCA7000800F012B8704700BF704700BFBD
S3150800549041F61C73C2F2000300221A709A6483F85C
S315080054A04320A3F844209A705A70704741F61C733B
S315080054B0C2F200031878003018BF0120704700BFF9
S315080054C041F61C73C2F20003002283F8432070479A
S315080054D0F8B50578FF2D064640D0AA4C2378012B4F
S315080054E000D0F8BDC93D352D00F28180DFE815F002
S315080054F087007F007F009B007F007F00C500A30018
S31508005500B800CD007F007F007F007F007F007F000E
S315080055107F007F007F007F007F007F007F007F0085
S315080055207F007F007F007F007F007F007F007F0075
S315080055307F007F007F007F007F007F007F007F0065
S315080055407F007F00DC000A0117012B017F007F0026
S315080055507F0033017F0042015201760000F0B0F966
S31508005560884C08BBFE2110230220E1702371A4F8A1
S31508005570440094F84320834B012A0DD0B3F8441015
S3150800558008B20028ADDD89B27F48012384F843308C
S31508005590BDE8F840FFF72CBF0221FE221020DA7082
S315080055A01871A3F84410EFE7002110230126617053
S315080055B0237161712670E570FFF744FFA071FFF74C
S315080055C051FFE071FFF74EFF0822000A207266724B
S315080055D0A672A4F84420FFF7EBFACAE70020FF21D9
S315080055E0012220706070E170A4F84420C1E7FE2310
S315080055F020200222E3702071A4F84420B9E7A76CA2
S31508005600604DFFF71FFF721C411E3846FFF7D2FA9E
S31508005610002840F0D180FE2031220221E8702A714C
S31508005620A5F84410A5E7FE2131230220E170237175
S31508005630A4F844009DE7FFF705FF73780138984200
S3150800564065DDFF250122E570A4F8442071784D4DEB
S31508005650002940F0BD80FFF7B5FA002889D1DAE7BE
S31508005660A06C7168474DFFF7A7FA0028D3D0FF2230
S315080056700121EA70A5F844107BE7FEF7A7FFFF2093
S315080056800122E070A4F8442073E70025FF20E070AB
S3150800569025716571FFF7D6FE0723A071E57125729E
S315080056A06572A4F8443064E7FF25E5704568A26C86
S315080056B0002D00F099801346D04313F8011BAD184E
S315080056C04219AB4202F0010011D028B113F8012BA0
S315080056D08918AB42C9B20AD01A465B7812F8010B90
S315080056E0091853FA81F0531CAB42C1B2F4D1002316
S315080056F0C4F807100122082122716371A371A4F866
S31508005700441036E7FFF79EFE727890424FDCFE2281
S3150800571022210223E2702171A4F8443029E7FFF719
S3150800572091FE72789042F2DD1848A16CFEF76EFF82
S31508005730FF20E0707178A36CCA18A2647078411CC7
S31508005740A4F8441015E7FF22E27043680121A36418
S31508005750A4F844100DE700200D4B2071FF2260715C
S31508005760A07107210820E270A364C4F80710A4F802
S315080057704400FEE6FE2000230221E0702371A4F80F
S315080057804410F6E61C1F00201F1F0020201F0020C3
S3150800579000A8000860780023FF210622E170237123
S315080057A06071A371E3712372A4F84420E1E671687D
S315080057B00E48A1647278B9E7FF22AE6CEA70FFF76B
S315080057C041FE013E31180123A964A5F84430D0E60C
S315080057D0A86CB21CFFF7EEF900283FF41CAF7178ED
S315080057E0AB6CC818A864C4E6294680E7201F0020C9
S315080057F038B50546007804F079FDC0B2A0F130044A
S31508005800E4B2162C1FD8A0F13A02062A1BD9092C95
S3150800581088BFA0F13704687888BFE4B204F066FD53
S31508005820C1B2A1F13003D8B216280CD8A1F13A02B8
S31508005830062A08D9092884BFA1F13700C0B200EBAF
S315080058400414E0B238BD002038BD00BF38B505469F
S31508005850000909280C460CD905F00F053730092D23
S3150800586020700FD905F1370000236070A370204619
S3150800587038BD303004F03AFD05F00F05C0B2092DE9
S315080058802070EFD805F1300004F030FDC0B2EBE728
S3150800589008B5074B0748084900221A7002F018FD98
S315080058A000B908BD05487721BDE80840FFF7ECBCFC
S315080058B0A81F0020B41F002008A800080CA800088C
S315080058C041F6A873C2F200031878D0F1010038BF78
S315080058D00020704710B5FFF7D5FD012802D0054C0A
S315080058E023780BB1002010BDFEF7A6FA0128F9D1DE
S315080058F0207010BDA81F002010B50446007804F0DB
S31508005900F5FC532801D0032010BD607804F0E6FCAE
S315080059100028F8D06078312806D0322806D03328F7
S3150800592014BF0320022010BD002010BD012010BDA9
S31508005930F8B507460230FFF75BFF0546381DFFF747
S3150800594057FF6C1EA4B2281805F00103BD1D012CD3
S31508005950C6B21DD953B12846FFF74AFF611E8CB25D
S315080059603218012CD6B207F1080511D92846FFF7D7
S315080059703FFF02353318013C2846DEB2A4B2FFF7D2
S3150800598037FF611E8CB230180235012CC6B2EDD82D
S315080059902846FFF72DFFF243D6B2331A594251EB88
S315080059A00300F8BD2DE9F0410F46054616460029C5
S315080059B039D0002837D02846FFF79EFF032804462B
S315080059C02DD02846FFF7B4FF002800F08F80012C61
S315080059D02FD022D2A81CFFF70BFF8046281DFFF701
S315080059E007FF04023C60A81DFFF702FFA8F10303A6
S315080059F0201899B2386008350CB28EB1002C0FDD2C
S31508005A0000272846FFF7F4FE7A1CF05597B20235B0
S31508005A10A742F6DB2046BDE8F081022C34D00024EC
S31508005A202046BDE8F081334840F26121FFF72CFC9F
S31508005A30C1E7A81CFFF7DCFE8046281DFFF7D8FE45
S31508005A4004043C60A81DFFF7D3FE04EB00243C6069
S31508005A5005F10800FFF7CCFEA8F10403201899B257
S31508005A6038600A350CB2002EDAD0002CD8DD0027B3
S31508005A702846FFF7BDFE7A1CF05597B20235A742B5
S31508005A80F6DB2046BDE8F081A81CFFF7B1FE80468C
S31508005A90281DFFF7ADFE04063C60A81DFFF7A8FE0B
S31508005AA004EB00443C6005F10800FFF7A1FE04EB97
S31508005AB000243C6005F10A00FFF79AFEA8F10503E9
S31508005AC0201899B238600C350CB2002EA8D0002CDC
S31508005AD0A6DD00272846FFF78BFE7A1CF05597B2FD
S31508005AE00235A742F6DB2046BDE8F0814FF0FF34C9
S31508005AF096E700BF0CA800082DE9F047A94D2C78B9
S31508005B003CB1012C00F02381022C00F09680032C76
S31508005B1001D0BDE8F087A44FA44E4FF480713046FB
S31508005B2007F50C7203F03EF897F84192B9F1000FA9
S31508005B3040F0838100285DD0304606F5C07106F531
S31508005B408072FFF72FFFB0F1FF3F804600F05C81BF
S31508005B5000284FDD9648FEF7D3F94CF6CD40954B15
S31508005B604446CCF6CC40A0FB041219460133D408AF
S31508005B70F9D14CF6CD400C700A464446CCF6CC40DA
S31508005B80A0FB0413DB0803EB8301A4EB410404F137
S31508005B90300102F8011D1C46002BF1D18648FEF79C
S31508005BA0AFF98648FEF7ACF9834996F88301FFF703
S31508005BB04DFE834996F88201FFF748FE814996F81B
S31508005BC08101FFF743FE804996F88001FFF73EFE04
S31508005BD07948FEF795F97D48FEF792F9D6F88001DF
S31508005BE07B4A4146FEF7E6FF002800F042817948E5
S31508005BF0FEF786F9D7F84402D7F83C22904288D1B6
S31508005C007548FEF77DF9FEF7DDFF0446002800F02B
S31508005C10A2817048FEF774F97048FEF771F970486A
S31508005C2002F066FE6F48FEF76BF900232B70FEF74D
S31508005C3039F9BDE8F047FEF7C9BC5B4E5B4F4FF438
S31508005C408071384606F50C7202F0ACFF96F8418270
S31508005C50B8F1000F40F0FF80B8B1384607F5C071BB
S31508005C604246FFF79FFEB0F1FF3F814600F07F8175
S31508005C7000280ADDDFF87081D8F80400002840F013
S31508005C80D180D7F8803188E80802D6F84422D6F8B9
S31508005C903C329A427FF43DAF5148002102F038FE6B
S31508005CA0002840F07281504E7168002948D0494852
S31508005CB0FEF726F94D48FEF723F974683D4B4CF676
S31508005CC0CD402246CCF6CC40A0FB02121946013341
S31508005CD0D208F9D14CF6CD400A70CCF6CC400A462B
S31508005CE0A0FB0413DB0803EB8301A4EB410130316D
S31508005CF01C4602F8011D002BF2D12F48FEF700F9C9
S31508005D003B48FEF7FDF82C49F078FFF79FFD2C4934
S31508005D10B078FFF79BFD2B497078FFF797FD2A4966
S31508005D203078FFF793FD2448FEF7EAF82748FEF790
S31508005D30E7F896E80300FEF73FFF002800F0FF802B
S31508005D402448FEF7DDF803202870BDE8F087FEF743
S31508005D502FFFFEF793F82748FEF7D2F82648FEF7F6
S31508005D60CFF8FEF785F8224601461D4802F0DCFA10
S31508005D70064638B12148FEF7C3F82046BDE8F04785
S31508005D80FEF7B4B81348FEF7BBF81D48FEF7B8F897
S31508005D901C48FEF7B5F8144902200E604E602870BC
S31508005DA0BDE8F087A81F0020B41F00200C2400209F
S31508005DB0A8A90008691F0020681F0020B8A90008C4
S31508005DC06A1F00206C1F00206E1F0020E8A900082B
S31508005DD00C250020DCA80008D0A90008ECA90008BA
S31508005DE0E421002004AA0008AC1F002038A90008F6
S31508005DF044A9000888A80008ACA80008D4A8000888
S31508005E00E4A8000808A900086648FEF779F82046BD
S31508005E10FEF76CF807F50C7002F06AFD85F800903D
S31508005E20BDE8F087D8F80030D7F88021C1188A4233
S31508005E302BD14844C8F8040027E75B48FEF760F80A
S31508005E400220FEF753F807F50C7002F051FD002109
S31508005E502970BDE8F0875548FEF752F82046FEF748
S31508005E6045F806F50C7002F043FD00232B70BDE8DB
S31508005E70F0874E48FEF744F80620FEF737F84C48F8
S31508005E8002F036FD2C70BDE8F0874A48FEF738F870
S31508005E904948FEF735F8D8F80440484B4CF6CD404B
S31508005EA02246CCF6CC40A0FB021219460133D20892
S31508005EB0F9D14CF6CD400A70CCF6CC400A46A0FB88
S31508005EC00413DB0803EB8301A4EB410404F130015E
S31508005ED002F8011D1C46002BF1D13948DFF8FCA059
S31508005EE0FEF70EF83748FEF70BF8354998F8030021
S31508005EF0FFF7ACFC344998F80200FFF7A7FC3349D2
S31508005F0098F80100FFF7A2FC314998F80000FFF75E
S31508005F109DFC2B48FDF7F4FF2E48FDF7F1FF98E8A6
S31508005F200300FEF749FE50B12248FDF7E9FF2A486B
S31508005F30FDF7E6FFD7F880318AE80802A5E61B4890
S31508005F40FDF7DEFF0520FDF7D1FF194802F0D0FC6A
S31508005F502C70BDE8F0871548FDF7D2FF0720FDF73E
S31508005F60C5FF134802F0C4FC2C70BDE8F0870F4843
S31508005F70FDF7C6FF0320FDF7B9FF06F50C7002F022
S31508005F80B7FC85F80080BDE8F0870848FDF7B8FF3C
S31508005F900420FDF7ABFF064802F0AAFC00222A708F
S31508005FA0BDE8F08784A9000860A90008D4A80008FD
S31508005FB0E4210020DCA8000838A90008691F002091
S31508005FC0681F002044A900086A1F00206C1F0020D3
S31508005FD06E1F0020E8A9000808A90008AC1F0020C9
S31508005FE0F0B404680646BCB125781F2D0BD93A2DA6
S31508005FF012D0671C3B4601E03A2A07D0194613F827
S31508006000012B1F2AF8D80020F0BC7047A5F13000F4
S31508006010092801D88F4202D04FF0FF30F4E7002854
S31508006020FAD102343460EFE710B5044682B018B1ED
S3150800603003680BB11A7822B900200860092002B05B
S3150800604010BDD888A2889042F6D158780191FBF7FE
S315080060507FF910F001000199EED123680B60EEE795
S3150800606030B401230D78541E9342057004EA0304E4
S315080060700DD024B14C7802239342447007D0CD5CEE
S315080060805C1CC55402330D5D93420555F7D130BCEF
S31508006090704700BF2DE9F843436A013306460D46AB
S315080060A030D0816A088848B3884600241EE0FF2C51
S315080060B024D0907537F8023F01341846A146F3B14B
S315080060C002F0BAFD2A190021C0B1907537F8023FCF
S315080060D0013418469BB102F0AFFD2C1970B1A075BA
S315080060E0788809F1020408F1060840B1002102F097
S315080060F0A3FD47462A1900210028D8D100242819CB
S3150800610000218175F269A97D1378202B00F054814E
S31508006110052B08BFE5236B72002900F03F81F26961
S3150800612001235078202809D0EA18052808BFE52059
S315080061305072002900F00881F2690133907820280E
S3150800614009D0EA18052808BFE5205072002900F092
S315080061501781F2690133D078202809D0EA18052872
S3150800616008BFE5205072002900F0D280F269013399
S315080061701079202809D0EA18052808BFE5205072AA
S31508006180002900F0B780F26901335079202809D038
S31508006190EA18052808BFE5205072002900F09C80FF
S315080061A0F26901339079202809D0EA18052808BF32
S315080061B0E5205072002900F08180F2690133D07918
S315080061C0202808D0EA18052808BFE52050720029BB
S315080061D066D0F2690133107A20281BD0052808BF3B
S315080061E0E520002953D15A1CAC18EB18A0F1410C34
S315080061F02E27BCF1190F5F729F75607207D8F36975
S315080062001B7B03F01003DBB20BB12030C0B2A075C4
S31508006210531CF269507A202809D0EA18052808BFC5
S31508006220E5205072002900F09D80F2690133927AC8
S31508006230202A07D0E818052A08BFE5224272002955
S3150800624074D00133E81829B98175F1690C7B002CE3
S3150800625008BF284600224272F369D87A2872F36981
S31508006260DC7F9A7F587F197F42EA042240EA02209F
S3150800627041EA00212960587E1A7E42EA0021A98057
S31508006280D87D9B7D43EA0022EA80BDE8F8835A1C44
S31508006290AC18EB182E275F726072531CF269B9E7C7
S315080062A0A0F14104192C07D8F469247B04F00804EA
S315080062B0E4B20CB12030C0B290758AE7A0F141046F
S315080062C0192C07D8F469247B04F00804E4B20CB14D
S315080062D02030C0B2907570E7A0F14104192C07D898
S315080062E0F469247B04F00804E4B20CB12030C0B28F
S315080062F0907555E7A0F14104192C07D8F469247B59
S3150800630004F00804E4B20CB12030C0B290753AE744
S31508006310A0F14104192C07D8F469247B04F0080479
S31508006320E4B20CB12030C0B290751FE7A2F1410467
S31508006330192C07D8F469247B04F01004E4B20CB1D4
S315080063402032D2B282757CE7A0F14104192C07D815
S31508006350F469247B04F00804E4B20CB12030C0B21E
S315080063609075E9E6A0F14104192C07D8F469247B55
S3150800637004F01004E4B20CB12030C0B2907554E7B2
S31508006380A0F14104192C07D8F469247B04F0080409
S31508006390E4B20CB12030C0B29075DAE6A3F141023E
S315080063A0192A07D8F469207B00F00802D4B20CB188
S315080063B02033DBB2AB75B2E60023B2E6F8B5044685
S315080063C0C07800B9F8BDE56A607804F13006314650
S315080063D02A460123FAF7FEFF18BB226AA369E07072
S315080063E0A81A98421BD2A778012F18D9FA070CD5F4
S315080063F0ED18607802E0A16960786D1801233146CE
S315080064002A46FAF7E7FFA369013FED18314601234B
S315080064102A466078013FFAF7DDFF012FEBD100200D
S31508006420F8BD0120F8BD00BF2DE9F04F83B0044642
S31508006430FFF7C4FF50B92378032B0AD000216078F0
S315080064400A46FAF7F7FF003018BF012003B0BDE887
S31508006450F08F21790129F1D104F1300104F50C7589
S315080064600E46324602F8010B7070561CAE42F8D141
S31508006470E368D4F81080E06984F81C324FEA136B9D
S31508006480CDF804B04FEA132C4FEA134E4FF0550BD4
S31508006490019B84F81882421C5227612041257226E6
S315080064A04FEA182A4FEA184984F82EB24FEA1868B4
S315080064B04FF0AA0B84F8320084F8170284F81F32CA
S315080064C084F82FB284F8307084F8317084F8335029
S315080064D084F8146284F8156284F8165284F819A2AE
S315080064E084F81A9284F81B8284F81DC284F81EE286
S315080064F0E26260780123FAF76DFF002121719DE7BA
S31508006500C36A8B4270B505460E4615D0FFF756FF8F
S31508006510044608B1204670BD32460123687805F165
S315080065203001FAF729FF002818BF4FF0FF3618BFC9
S315080065300124EE62204670BD0024204670BD00BFCF
S315080065400129F8B50C46056809D96B69994206D23E
S31508006550287802282ED0032810D0012801D001203F
S31508006560F8BD296A04EB5406284601EB5621FFF7C5
S31508006570C7FF002831D04FF0FF30F8BD2B6A2846F8
S3150800658003EBD111FFF7BCFF0028F4D16406E00D38
S3150800659000F13002AB182C189978D8785A7894F804
S315080065A0303041EA002042EA002143EA012222F083
S315080065B07040F8BD2B6A284603EB1121FFF7A0FFB0
S315080065C00028D8D12406E00D29180C4691F8302069
S315080065D091F8313042EA0320F8BDF205D70D296A51
S315080065E0EB190136284601EB562193F83070FFF770
S315080065F087FF0028BFD1F605F60DAD19E10795F816
S31508006600300047EA002201D51009F8BD1105080D2A
S31508006610F8BD00BFB1F5001FF8B505460C4606687B
S3150800662001D30220F8BDCB06FBD18168046129B9E4
S315080066303378022B18D9726AB2B1114677897F026C
S31508006640BC4207D223E00129EBD973699942E8D203
S31508006650A7421DD82846FFF773FF01460130C7EB4E
S315080066600404F0D10120F8BD3089B0EB541FD8D905
S31508006670736AAB616961002BD3D0E105CA0D30326C
S3150800668003EB5423B618AB61EE610020F8BD7369BD
S31508006690023B8A1E9A423DBF7089B36A00FB0233E9
S315080066A00023AB61E6E700BF38B54FF0FF320023A1
S315080066B0C370C2620446FFF723FF08B1042038BD41
S315080066C094F82E2294F82F124AF6552342EA01210D
S315080066D00AB2CFF6FF739A4201D0032038BD94F868
S315080066E0695094F8682094F8671094F8663042EA7E
S315080066F0052241EA022143EA012244F2461322F026
S315080067007F41C0F254039942E8D094F8855094F832
S31508006710840094F8831094F8822040EA052041EA20
S31508006720002142EA012222F07F40984214BF02204B
S31508006730002038BD2DE9F041002384B00B600D46DA
S315080067401746FFF74DFC061E19DBB14850F82640E0
S31508006750BCB12C60217807F0FE0721B16078FAF702
S31508006760F7FDC2070FD50022F0B222706070FAF763
S31508006770D7FDC30712D5032004B0BDE8F0810B206E
S31508006780FAE70C20F8E7002F00F0208100F004005B
S31508006790C1B2002914BF0A200020EDE72FB100F08E
S315080067A00403D8B208B10A20E6E700212046FFF71D
S315080067B07BFF022807D00025042800F0098101285C
S315080067C064D90D20D8E794F8F251002D00F006811F
S315080067D094F8F90194F8F85194F8F72194F8F631F9
S315080067E045EA002142EA012043EA002194F80252D0
S315080067F00091002D00F0F08094F8090294F8081230
S3150800680094F8075294F8063241EA002245EA022033
S3150800681043EA002294F812120192002900F0DA8065
S3150800682094F8190294F8181294F8172294F8163264
S3150800683041EA002542EA052043EA002594F8221297
S31508006840029569B194F8295294F8281294F82722E7
S3150800685094F8263241EA052042EA002543EA052152
S31508006860009D0391002D40F0BB80019D002D40F056
S31508006870BF80029D002D40F0C380039D002DA0D04F
S3150800688020462946FFF710FF012895D894F83C20A2
S3150800689094F83B3043EA0220B0F5007F91D194F892
S315080068A0471094F8462052EA01220DD194F8561062
S315080068B094F8570094F8552094F8543041EA00208B
S315080068C042EA002143EA012294F84000A261431EED
S315080068D0012BA0703FF675AF94F83D306381002B0D
S315080068E03FF46FAF591E19427FF46BAF94F841100D
S315080068F094F8426041EA0626B1B216F00F0F2181DC
S315080069007FF45FAF94F8447094F8436056EA07261C
S315080069100DD194F8538094F852C094F8517094F8B5
S3150800692050604CEA082E47EA0E2746EA072694F8EE
S315080069303FC094F83E7057EA0C273FF442AF00FB7D
S3150800694002FE07EB111070448642FFF43AAF361A7E
S31508006950B6FBF3F3002B3FF434AF40F6F576B342BB
S3150800696040F2E38006F57046B34200F2BA8002268A
S315080069700233EF1940196361E5612762A0620029B5
S315080069803FF41FAF7744022E676200F0A880032108
S3150800699001FB03F603F0010303EB5600012600F2A0
S315080069A0FF13B2EB532FFFF40CAF4FF0FF328020EA
S315080069B0032E2261E26020712ED0164826700188C7
S315080069C04A1C93B20380E3800020D5E63846D3E616
S315080069D00120D1E60D4631E72A461BE7294605E799
S315080069E020462946FFF760FE01283FF63EAF4DE7F1
S315080069F020462946FFF758FE01283FF63AAF45E7F5
S31508006A0020462946FFF750FE01283FF636AF3DE7F8
S31508006A10942700209027002094F8611094F860309D
S31508006A2043EA0122012AC8D12046691CFFF768FDFE
S31508006A300028C2D194F82F1294F82E32207143EA16
S31508006A4001204AF6552102B2CFF6FF718A42B4D127
S31508006A5094F8321094F8330094F8313094F83020D2
S31508006A6041EA002043EA002145F2522342EA012284
S31508006A70C4F261139A42A0D194F8161294F8170238
S31508006A8094F8153294F8142241EA002043EA0021CA
S31508006A9047F2722342EA0122C6F241139A428CD186
S31508006AA094F81B8294F81A7294F81FE294F81E520E
S31508006AB094F8190294F81D1294F8182294F81C32C6
S31508006AC047EA082745EA0E2540EA072041EA052154
S31508006AD042EA002243EA01232261E3606DE7580097
S31508006AE05DE794F85BC094F85A60E5610233EF19E4
S31508006AF0401956EA0C2663612762A0627FF461AEEC
S31508006B0000297FF45EAE94F85F7094F85E6094F89E
S31508006B105D0094F85C1046EA072640EA062041EA3A
S31508006B20002161629800032639E7012620E700BFA5
S31508006B30F0B5012983B00C46054602D94369994246
S31508006B4002D3022003B0F0BD0178022958D00329E8
S31508006B5035D00129F5D1036A019204EB540603EBFB
S31508006B605621FFF7CDFC019A0028EBD1F005C10D9F
S31508006B70013614F0010459D06B18D0B293F83010CE
S31508006B8001F00F0141EA0010C0B2296A83F830000B
S31508006B900123EB70284601EB56210192FFF7B0FC62
S31508006BA0019A0028CED1F605F10D002C41D0C2F38A
S31508006BB007126E18012386F83020EB70C2E7016AC7
S31508006BC0019201EBD411FFF79BFC019A0028B9D179
S31508006BD06406E70D07F13006AB1922F07042D97842
S31508006BE00C0604F070463243EC19160C170A110EFF
S31508006BF084F830205F709E70D9700123EB70A1E78E
S31508006C00016A019201EB1421FFF77AFC019A002828
S31508006C1098D12406E30DE918C2F3072381F830203A
S31508006C20012281F831300C46EA708BE7D0B26B1836
S31508006C30ABE76E18C2F3032296F8303023F00F0143
S31508006C400A43B7E72DE9F04107468846066809BBB7
S31508006C50F5687369CDB19D4228BF01252C460134DC
S31508006C609C4202D3012D12D9022438462146FFF749
S31508006C7067FCD0B1012825D001301FD0AC4206D020
S31508006C80736901349C42EDD2EFE70125E6E700205F
S31508006C90BDE8F081FFF754FC012813D9411C0DD03B
S31508006CA0736998420FD34546D8E7304621464FF0D8
S31508006CB0FF32FFF73DFF40B1012803D14FF0FF3007
S31508006CC0BDE8F0810120BDE8F081B8F1000F0ED1D2
S31508006CD072693069F460911E884201D2431E33619D
S31508006CE0327942F0010030712046BDE8F081304625
S31508006CF041462246FFF71CFF0028E9D0DCE700BF23
S31508006D002DE9F04783690568026982B004460E4694
S31508006D101BB9042002B0BDE8F08702F12007B7F5D9
S31508006D20001FF6D2F905CA0D1ABB41690133836102
S31508006D3029B36B89013B13EA57231AD10192FFF74E
S31508006D40FFFB01288046019A20D9B0F1FF3F23D0E6
S31508006D50686980451CD2A8F10206831E9E423CBF84
S31508006D606989AB6AC4F8148034BF01FB063600266D
S31508006D70A6613032AD182761E5610020CAE72B8984
S31508006D80B3EB571FF5D881610420C3E70220C1E79A
S31508006D9026B9A6610420BDE70120BBE76169019217
S31508006DA02046FFF74FFF804608B90720B2E70128BB
S31508006DB0ECD0B0F1FF3FEFD02846FFF7FFFA019A73
S31508006DC00028E9D105F1300305F50C76194601F8D6
S31508006DD0010B58704B1CB342F8D16869A8F102063A
S31508006DE0831E9E4238BFA96A6B8934BF03FB06110E
S31508006DF00021E9624FF000094FF0010A0DE085F81D
S31508006E0003A00192FFF7DAFA019A0028C4D1E96AC9
S31508006E106B89481C09F10109E86299452846EED3B1
S31508006E20E96A6869C9EB0101E96296E72DE9F04F5D
S31508006E30002187B083460668FFF7ECFB002840F080
S31508006E40CD80FF224FF0FF330292CBF8243015464F
S31508006E500EE00F2A00F0C5804FF0FF30CBF8240073
S31508006E60FF2558460021FFF74BFF002840F0B68063
S31508006E703046DBF81810FFF743FB002840F0AE80D9
S31508006E80DBF81C402378002B00F0C780E17AE52B5D
S31508006E9001F03F028BF80620DED001F00801C9B2E6
S31508006EA00029D6D10F2A00F09C80002D59D12378CD
S31508006EB094F8019094F8028094F803C027796579CC
S31508006EC0A27903954FEAC31A4AEA530303EB090E5C
S31508006ED05FFA8EF94FEAC91343EA590958FA89F84D
S31508006EE05FFA88FE4FEACE1343EA5E085CFA88FC2E
S31508006EF05FFA8CFE4FEACE1343EA5E0C57FA8CF71C
S31508006F00FFB2FB0143EA5703039F049257FA83F340
S31508006F10DBB2DF0147EA5303049FE179257A05913D
S31508006F2057FA83F3DBB2DF0147EA5303059F617A19
S31508006F30A27A57FA83F3DBB2DF0147EA530355FA1D
S31508006F4083F5EDB2EB0143EA550551FA85F1C9B26D
S31508006F50CB0143EA510152FA81F2029BD1B28B422C
S31508006F603CD0DBF82030DA7AD2072BD421781A788D
S31508006F70914227D161785A78914223D1A1789A789B
S31508006F8091421FD1E178DA7891421BD121791A7999
S31508006F90914217D161795A79914213D1A1799A7997
S31508006FA091420FD1E179DA7991420BD1217A1A7A95
S31508006FB0914207D1617A5A7A914203D1A17A9B7A92
S31508006FC099420BD04FF0FF37CBF824705846002172
S31508006FD0FF25FFF795FE00283FF44AAF07B0BDE846
S31508006FE0F08FDBF82870002F3FF43BAF03F040002A
S31508006FF0C2B272B1DBF81050617BCBF82450029113
S3150800700003F0BF0594F80D90029B994507D0FF251C
S3150800701027E79D42F6D0FF2523E70420DEE7E07E3A
S31508007020A27E52EA002340F0D9812378A1786078BD
S3150800703003F03F02531E03EB430A03EB8A0ABAF135
S31508007040FE0F40EA012100F2C9810846019101F0CC
S315080070501BFE024637F81A00009201F015FE009B47
S3150800706083420AF10108019840F0B8812179E27853
S3150800707042EA0123002840F08D804FF6FF708342D4
S3150800708040F0AC81A179627942EA01214FF6FF729C
S31508007090914240F0A381207AE17941EA00234FF634
S315080070A0FF718B4240F09A81A07A627A42EA002107
S315080070B04FF6FF72914240F09181E07BA17B41EA55
S315080070C000234FF6FF718B4240F08881607C227C5A
S315080070D042EA00214FF6FF72914240F07F81E07C40
S315080070E0A17C41EA00234FF6FF718B4240F076817E
S315080070F0607D227D42EA00214FF6FF72914240F000
S315080071006D81E07DA17D41EA00234FF6FF718B4238
S3150800711040F06481607E227E42EA00214FF6FF72CB
S31508007120914240F05B81607F217F41EA00234FF660
S31508007130FF718B4240F05281002094F81FE0A17F36
S3150800714041EA0E2A002800F04D81B8F1FF0F00F041
S315080071504581504601F098FD034637F8180000931C
S3150800716001F092FD0099814208F1010840F036814C
S31508007170207800F04002D3B23BB1BAF1000F04D038
S3150800718037F81810002940F02981013DEDB2CDF8F5
S31508007190089066E6B8F1FF0F00F0208118460093C4
S315080071A001F072FD034637F81800019301F06CFDF3
S315080071B0019A82420AF10208009840F00F81A179EB
S315080071C0637943EA012100283FF460AFB8F1FF0F65
S315080071D000F004810846019101F056FD024637F891
S315080071E01800009201F050FD009981420AF1030847
S315080071F0019840F0F380227AE37943EA02230028D3
S315080072003FF44DAFB8F1FF0F00F0E8801846009341
S3150800721001F03AFD034637F81800019301F034FDF2
S31508007220019A82420AF10408009840F0D780A17AB0
S31508007230637A43EA012100283FF43AAFB8F1FF0F19
S3150800724000F0CC800846019101F01EFD024637F891
S315080072501800009201F018FD009981420AF105080C
S31508007260019840F0BB80E27BA37B43EA0223002817
S315080072703FF427AFB8F1FF0F00F0B080184600932F
S3150800728001F002FD034637F81800019301F0FCFCF3
S31508007290019A82420AF10608009840F09F80617CB4
S315080072A0237C43EA012100283FF414AFB8F1FF0F0D
S315080072B000F094800846019101F0E6FC024637F892
S315080072C01800009201F0E0FC009981420AF10708D3
S315080072D0019840F08380E27CA37C43EA02230028DD
S315080072E03FF401AFB8F1FF0F78D01846009301F0CC
S315080072F0CBFC034637F81800019301F0C5FC019A48
S3150800730082420AF10808009868D1617D237D43EA24
S31508007310012100283FF4F0AEB8F1FF0F5ED0084611
S31508007320019101F0B1FC024637F81800009201F00D
S31508007330ABFC009981420AF1090801984ED1E27D19
S31508007340A37D43EA022300283FF4DFAEB8F1FF0F1E
S3150800735044D01846009301F097FC034637F8180006
S31508007360019301F091FC019A82420AF10A080098F9
S3150800737034D1617E237E43EA012100283FF4CEAE54
S31508007380B8F1FF0F2AD00846019101F07DFC0246AC
S3150800739037F81800009201F077FC009981420AF14B
S315080073A00B0801981AD1627F237F43EA022300283B
S315080073B03FF4BDAEB8F1FF0F10D01846009301F0A8
S315080073C063FC024637F81800019201F05DFC019B48
S315080073D083420AF10C0800983FF4AFAECDF8089046
S315080073E0FF253EE54FF6FF7292453FF4CEAEF5E730
S315080073F02DE9F04FD0F800B085B007460D460131AB
S315080074002B782F2BFAD05C2BF8D00021B96028787E
S315080074101F2840F284814FF0200A1F28BE6A2FD900
S315080074202F282DD05C282BD00121A6F10209A846C9
S31508007430012401F001FCF8B17F2809D822281BD0C5
S31508007440B04A01E0884217D012F8011F0029F9D185
S3150800745029F8020F18F8010F631C1F2812D92F28C4
S3150800746010D05C280ED0B3F5807F05D001211C46CC
S3150800747001F0E2FB0028DFD1062005B0BDE8F08F59
S3150800748000240123E9180D4601312A782F2AFAD05B
S315080074905C2AF8D01F2894BF4FF004094FF0000962
S315080074A02CB306EB4400631E30F8022D202A03F0A5
S315080074B0010101D02E2A1ED1013C18D039B130F86D
S315080074C0023D202B01D02E2B15D1013C0FD030F8D0
S315080074D0022D202A01D02E2A0DD130F8021D013C9A
S315080074E02029234601D02E2905D15C1EEFD1002084
S315080074F0B0463080C0E73A6A002126F81410B31E59
S3150800750006EB440182F800A082F801A082F802A0E6
S3150800751082F803A082F804A082F805A082F806A0E3
S3150800752082F807A082F808A082F809A082F80AA0C3
S315080075304FF0000801E008F1010833F8020F20288F
S31508007540F9D02E28F7D0B8F1000F01D049F0030979
S315080075500B46621E33F802EDBEF12E0F02F0010152
S3150800756012D0144682B121B133F8022D2E2A09D140
S315080075700AE033F8021D2E2906D033F8022D013C05
S315080075802E2A01D0013CF4D1002221469446144605
S3150800759008232A4635460E4608F1010878B32028FE
S315080075A01FD02E281BD09C4220D2464576D07F2855
S315080075B07ED82B2800F09480DFF84CE102E0884260
S315080075C000F08E801EF8011F0029F8D1A0F14101B4
S315080075D0192900F29B804CF0020CC0B283E04645A4
S315080075E05CD049F0030935F81800D5E70B2B00F0F5
S315080075F0AB80464554D0B04549F0030950D91546E5
S315080076003A6A1078E52875D0082B04BF4FEA8C0C27
S315080076105FFA8CFC0CF00C030C2B68D00CF0030002
S31508007620032864D009F00201C8B250B90CF0030E61
S31508007630BEF1010F08BF49F01009042B08BF49F035
S31508007640080982F80B903846FFF7F0FB3A6AD37AB6
S3150800765000286FD103F00401CAB2002A7FF40DAFE7
S31508007660B87900F01003D9B2002961D03E699BF8B9
S315080076700040F205D00D30300BEB0003032CD97E09
S315080076809E7E46EA012202D0BA602878C5E65C7D6D
S31508007690187D40EA042342EA0342F5E70B2B53D050
S315080076A04FEA8C045FFA84FCB0460B2308249AE759
S315080076B0002102920193CDF80CC001F0BDFA029A9E
S315080076C0019BDDF80CC0C8B14AF64421C0F600019A
S315080076D0081849F0020910F8800C00287FF469AFF1
S315080076E049F003095F20396A085501347BE749F0F8
S315080076F0020997E7052111703A6A85E749F00209F8
S31508007700EEE700BF30AA00083CAA0008A0F1610114
S31508007710192902D820384CF0010CC0B2E3E7386AC0
S315080077208022C272384605B0BDE8F04FFEF772BF38
S315080077300520A2E604287FF4A0AE03F00401CBB22C
S31508007740002B08BF052098E6154649F003090B23C8
S3150800775056E700BF416A4B1C2DE9F041044605680F
S31508007760066906D0FEF756FF034610B11846BDE86F
S31508007770F0814FF0E5080127A1692846FEF7C0FE0B
S315080077800346014620465BB9E26982F80080EF703D
S3150800779022699642EAD9FFF7B3FA03460028EBD0E6
S315080077A0042B08BF02231846BDE8F081012970B5ED
S315080077B006460C46056802D96B69994201D3022030
S315080077C070BD02BB21463046FEF7BAFE0346214687
S315080077D000220446284693B1012BF0D0013310D07D
S315080077E0FFF7A6F970B92869421C05D02A79411C09
S315080077F042F0010329612B7168698442E2D30020B3
S3150800780070BD012070BD114628464FF0FF32FFF7C4
S315080078108FF90028D6D0F5E72DE9F04FFF25044665
S31508007820076883B02E4604204FF000094FF6FF780C
S31508007830A169002900F0BF803846FEF761FEC0B98D
S31508007840E2691378002B00F0BA80D17AE52B01F0B3
S315080078503F01A17106D02E2B04D021F0200CBCF1DB
S31508007860080F0BD1FF2620460021FFF749FA00280A
S31508007870DED00021A16103B0BDE8F08F0F2940F0EA
S31508007880A58003F04000C1B2002900F09080266967
S31508007890557B666203F0BF03517BA942E2D1D67ECF
S315080078A0907EA56A50EA062040F08D80167892F8F8
S315080078B002C092F801E006F03F00013800EB4006EE
S315080078C000EB8606FE2E4EEA0C2E7CD825F816E02E
S315080078D092F804A092F803C0701C4CEA0A2ABEF17A
S315080078E0000F40F0D480C2456DD192F806E0567973
S315080078F046EA0E2CC44566D192F808C0D67946EAFF
S315080079000C2EC6455FD192F80AC0567A46EA0C2C68
S31508007910C44558D192F80FE0967B46EA0E2EC64526
S3150800792051D192F811C0167C46EA0C2CC4454AD1AE
S3150800793092F813E0967C46EA0E2EC64543D192F895
S3150800794015C0167D46EA0C2CC4453CD192F817E0C2
S31508007950967D46EA0E2EC64535D192F819C0167E92
S3150800796046EA0C2CC4452ED192F81DE0167F46EA4D
S315080079700E2EC64527D14FF0000E92F81FC0967FEF
S3150800798046EA0C26BEF1000F1BD0FF281BD025F8AF
S3150800799010600130127802F04006F2B21AB1FF28E0
S315080079A011D025F81090013BDEB20D465BE7B342D5
S315080079B07FF458AF70E700283FF45DAF59E704201D
S315080079C057E74645E6D00D46FF264CE7002E5AD126
S315080079D0137892F808B092F801A0CDF800B04FEAF3
S315080079E0C31B4BEA53035344DBB292F8029092F856
S315080079F0038092F804E057799679D17992F809C00C
S31508007A00927ACDF804C04FEAC31A4AEA530359FAE0
S31508007A1083F3DBB24FEAC31949EA530358FA83F3EF
S31508007A20DBB24FEAC31848EA53035EFA83F3DBB2C4
S31508007A304FEAC31E4EEA530357FA83F7FBB2DF0138
S31508007A4047EA530356FA83F6F3B2DE0146EA5303CE
S31508007A5051FA83F1CBB2D90141EA53030099DDF813
S31508007A6004B051FA83F3DBB2D90141EA53035BFA56
S31508007A7083F1CBB2D90141EA530352FA83F2D1B268
S31508007A80A9423FF4F8AE4FF0FF336362F3E6FF28EE
S31508007A9099D025F810A092F806C092F805E0B01C17
S31508007AA04EEA0C2CBAF1000F3FF424AFFF288AD017
S31508007AB025F810C092F808A092F807E0F01C4EEAE4
S31508007AC00A2EBCF1000F3FF41CAFFF283FF47BAF32
S31508007AD025F810E092F80AA092F809C0301D4CEA81
S31508007AE00A2CBEF1000F3FF413AFFF283FF46BAF2B
S31508007AF025F810C092F80FA092F80EE0701D4EEA15
S31508007B000A2EBCF1000F3FF40AAFFF283FF45BAF23
S31508007B1025F810E092F811A092F810C0B01D4CEAB2
S31508007B200A2CBEF1000F3FF401AFFF283FF44BAF1C
S31508007B3025F810C092F813A092F812E0F01D4EEA4C
S31508007B400A2EBCF1000F3FF4F8AEFF283FF43BAF16
S31508007B5025F810E092F815A092F814C006F108006E
S31508007B604CEA0A2CBEF1000F3FF4EEAEFF283FF4B4
S31508007B702AAF25F810C092F817A092F816E006F179
S31508007B8009004EEA0A2EBCF1000F3FF4E4AEFF28C6
S31508007B903FF419AF25F810E092F819A092F818C02A
S31508007BA006F10A004CEA0A2CBEF1000F3FF4DAAEE1
S31508007BB0FF283FF408AF25F810C092F81DA092F8E8
S31508007BC01CE006F10B004EEA0A2EBCF1000F3FF44A
S31508007BD0D0AEFF283FF4F7AE25F810E006F10C000A
S31508007BE0CBE600BF2DE9F04F066A0568F37AD0F8B0
S31508007BF0289013F0A00289B0044604D0062318463C
S31508007C0009B0BDE8F08FB9F8007037B14846174695
S31508007C1030F8021F01370029FAD105A831460C228F
S31508007C20FEF71EFA9DF81F00C10740F16881002380
S31508007C30F3723046A36205A90B224FF0010BFEF73B
S31508007C400FFA0DF10C0A5B464FF07E08072203F087
S31508007C500F0000F13001392988BF00F137010AF811
S31508007C600210013A1B09F2D108A8811801F8148CF0
S31508007C70002A00F0A0813078202815D0D007314698
S31508007C800FD43146012311F8010F202809D10BE042
S31508007C9011F8010F202807D011F8010F0133202809
S31508007CA002D001339342F3D1C3F10701072A01F049
S31508007CB0010000F2128108A98918013211F814ECA2
S31508007CC0591C072906F803E02FD810B3072A00F233
S31508007CD0098108A88318013213F8143C735401313A
S31508007CE0072916D921E00DF1200C0CEB020301320D
S31508007CF013F8140C4B1C072A705411D80DF1200EDA
S31508007D000EEB0201013211F8140C591C0729F05424
S31508007D100BD8072AE7D920204B1C072A7054EDD91F
S31508007D20591C20200729F054F3D92046FFF77EF87E
S31508007D30002840F0D9800BF1010BBBF1640F00F06D
S31508007D40C2820B22304605A9FEF78AF9BBF1050F58
S31508007D5040F2C680A9F102015B46B8E002F00100D4
S31508007D6000EB43035008DA0348BF83F4883300F076
S31508007D70010248BF83F0210302EB43034008DA03FC
S31508007D8048BF83F4883300F0010248BF83F021031B
S31508007D9002EB43034008DA0348BF83F4883300F054
S31508007DA0010248BF83F0210302EB43034008DA03CC
S31508007DB048BF83F4883300F0010248BF83F02103EB
S31508007DC002EB43034008DA0348BF83F4883300F024
S31508007DD0010248BF83F0210302EB43034008DA039C
S31508007DE048BF83F4883300F0010248BF83F02103BB
S31508007DF002EB43034008DA0348BF83F4883300F0F4
S31508007E00010248BF83F0210302EB43034008DA036B
S31508007E1048BF83F4883300F0010248BF83F021038A
S31508007E2002EB43034008DA0348BF83F4883300F0C3
S31508007E30010248BF83F0210302EB43034008DA033B
S31508007E4048BF83F4883300F0010248BF83F021035A
S31508007E5002EB43034008DA0348BF83F4883300F093
S31508007E60010248BF83F0210302EB43034008DA030B
S31508007E7048BF83F4883300F0010248BF83F021032A
S31508007E8002EB43034008DA0344BF83F4883383F0E4
S31508007E90210300F0010202EB43024308D00344BF6A
S31508007EA082F4883282F0210203F0010000EB4202DC
S31508007EB05B08D00344BF82F4883282F0210203EBC8
S31508007EC04203DA0344BF83F4883383F0210331F88D
S31508007ED0022F002A7FF442AFB8E64FF0200EEFE6F5
S31508007EE05B46B3E62023F9E6042803467FF487AE0B
S31508007EF09DF81F10F1729DF81F00C4F8289000F035
S31508007F000206F2B2002A48D1012620460021D4F8FA
S31508007F100080FEF77FFB0346002848D1074605E0A8
S31508007F201F46FEF7EDFE0346002840D1A1694046EC
S31508007F30FEF7E6FA0346013701212046002B36D123
S31508007F40E2691278E52A01D0002AE9D1BE42E8D1D1
S31508007F50013E32D12846A169FEF7D2FA0346002827
S31508007F607FF44DAEE269184602F12006114601F883
S31508007F70010B50704A1CB242F8D1E069216A00939D
S31508007F800B22FEF76DF8236AE069D97A012301F01E
S31508007F9018020273EB70009B31E64EF64F430C371E
S31508007FA0C4F6C463A3FB07018808461CADE7042B87
S31508007FB008BF072323E6134676E623692046A3EB84
S31508007FC04611FEF727FB034600287FF418AED4F8BF
S31508007FD020B09BF800309BF801A09BF802909BF814
S31508007FE003809BF804C09BF805E09BF806709BF895
S31508007FF007009BF808109BF809209BF80AB0CDF8F3
S3150800800004B04FEAC31B4BEA53035344DBB24FEAAF
S31508008010C31A4AEA530359FA83F3DBB24FEAC31980
S3150800802049EA530358FA83F3DBB24FEAC31848EA1E
S3150800803053035CFA83F3DBB24FEAC31C4CEA5303DF
S315080080405EFA83F3DBB24FEAC31E4EEA530357FACE
S3150800805083F7FBB2DF0147EA530350FA83F0C7B24E
S31508008060FB0143EA570051FA80F1CFB2FB0143EA1C
S31508008070570052FA80F2D1B2CF01019847EA51036C
S3150800808050FA83FA5FFA8AF94FF00F08FF274FF67E
S31508008090FF7A7DE0DF701F714FF6FF70504500F0E4
S315080080A0AB8031F812004FEA102C0132587183F870
S315080080B006C0002840F0A480DF711F724FF6FF70DB
S315080080C0504500F0AB8031F812004FEA102C01320F
S315080080D0587283F80AC0002840F0A4809F73DF73A3
S315080080E04FF6FF70504500F0AB8031F812004FEAAA
S315080080F0102C0132187483F811C0002840F0A480AF
S315080081009F74DF744FF6FF70504500F0AB8031F86E
S3150800811012004FEA102C0132187583F815C0002892
S3150800812040F0A4809F75DF754FF6FF70504500F04C
S31508008130AB8031F812004FEA102C0132187683F81A
S3150800814019C0002840F0A4801F775F774FF6FF70AC
S31508008150504500F0AB8031F812004FEA102C01327E
S31508008160987783F81FC0002840F0A48046F0400E98
S315080081705FFA8EFE83F800E001232046EB700021AB
S31508008180FEF7BEFD002840F0A080013E3FF4E2AEB7
S315080081902846A169FEF7B4F90246002A40F0958000
S315080081A05FFA86FE0EF1FF30E369A16A1A7300EBE7
S315080081B0400B00EB8B0C9A76DA7683F80D9083F8F1
S315080081C00B8031F81C004FEA102B0CF10102587095
S315080081D083F802B000283FF45DAF50453FF45AAF2C
S315080081E031F812004FEA102B0CF10202D87083F80E
S315080081F004B000287FF452AF5F719F714FF6FF708D
S3150800820050453FF459AF31F812004FEA102C0132AD
S31508008210D87183F808C000287FF452AF5F729F7246
S315080082204FF6FF7050453FF459AF31F812004FEA48
S31508008230102C0132987383F80FC000287FF452AFD0
S315080082401F745F744FF6FF7050453FF459AF31F80D
S3150800825012004FEA102C0132987483F813C00028D4
S315080082607FF452AF1F755F754FF6FF7050453FF4A8
S3150800827059AF31F812004FEA102C0132987583F87D
S3150800828017C000287FF452AF1F765F764FF6FF704F
S3150800829050453FF459AF31F812004FEA102C01321D
S315080082A0187783F81DC000287FF452AF9F77DF77D1
S315080082B04FF6FF7050453FF459AF31F812100029B8
S315080082C03FF454AF56E7072399E4034697E400BF03
S315080082D030B585B004AB019043F8041D18460091EB
S315080082E01546FDF77DFE002810DB0E4C54F82010CD
S315080082F009B100220A70019B53B10022012D1A70A0
S3150800830044F8203008D0104605B030BD0B20FBE7F6
S3150800831044F820301846F7E7684601A9FEF70AFA36
S31508008320F2E700BF942700202DE9F04192B00546F8
S315080083300191164670B1002302F01F07036003A9D6
S3150800834001A83A46FEF7F6F9044628B1204612B0C7
S31508008350BDE8F0810924F9E703985E4B079004AA63
S3150800836001990F9207A81193FFF742F830B116F05A
S315080083701C0F01D004284BD00446E7E70F9991F962
S315080083800B000028C0F2998016F01C0F35D19DF815
S31508008390223003F01002D1B2002940F0908006F096
S315080083A00200C2B20AB1D8077ED406F00806F3B2B4
S315080083B0039E0BB147F020070E9BF06A6B6228629A
S315080083C03178D87E9A7E032942EA00226ED0AA60C6
S315080083D093F81FC0997F5A7F187F2F74002341EAAC
S315080083E00C216B7442EA0121F2886B6140EA012094
S315080083F0E860EB612E60AA80A8E79DF8221011F0CC
S31508008400110F51D106F00400C6B246B108249DE703
S3150800841007A8FFF7E7FB47F008070028ACD107F0E5
S315080084200802D6B2002E4CD00E9B039E0022612075
S3150800843048219A73DA73597418740E9B9A75DA750B
S31508008440597618760E982022C2720E9B327893F8C7
S315080084501B80997E032A41EA082834D000209876A2
S31508008460D8763278032A04BF187558750E9B0022F1
S3150800847001211A775A779A77DA77F170B8F1000FEF
S3150800848098D007A84146F66AFFF790F900287FF4C6
S3150800849073AF31460398FEF733F8039E08F1FF32AF
S315080084A0F260002886D067E707244FE7587D197DD4
S315080084B041EA002042EA004289E7062446E7042406
S315080084C044E7039E78E7587D1A7D42EA002148EA88
S315080084D00148C3E7902500202DE9F04F994685B05D
S315080084E000238B46C9F8003003A904461546FDF754
S315080084F09BFD074628B9677C1FB9207CC10704D4B1
S315080085000727384605B0BDE8F08F6069E1680A1AA2
S31508008510954234BFA8469046B8F1000FF1D004F151
S31508008520280AC505ED0D002D2ED103994B895A1E33
S3150800853012EA502341D0A0694A690238023A9042A9
S3150800854049D302276774DCE7E269B24218D0237C74
S3150800855003F04000C3B25BB1487801235146F8F7EF
S3150800856039FF002858D1227C039922F04000207454
S315080085704878324651460123F8F7FEFE00284BD1CB
S315080085806569E661EE05F50DC5F50076464528BF31
S31508008590464605F128035846E1183246FDF760FDC0
S315080085A06269D9F80010B0188B19B8EB0608606133
S315080085B0B344C9F80030B4D1A3E700282FD1A06886
S315080085C00128BED9421C27D00399A0614A690238FE
S315080085D0023A9042B5D24A898E6A02FB0066002E9C
S315080085E0AFD05FEA58251E44AED05819904288BFCE
S315080085F0C3EB02054878324659462B46F8F7BCFEC7
S3150800860050B9227C02F04001CBB21BB1E069861B4F
S31508008610B5420BD86E02C3E70127677471E7A169F3
S3150800862001932046FDF78CFF019BC9E70BEB46201B
S3150800863051464FF40072FDF713FD6E02B0E700BF16
S315080086402DE9F04F994685B000238B46C9F80030CE
S3150800865003A904461746FDF7E7FC804658B994F87F
S315080086601180B8F1000F06D1217C01F00202D0B2C8
S3150800867028B94FF00708404605B0BDE8F08F626993
S31508008680D74228BFD743002F57D004F128010191BC
S31508008690D505ED0D002D2FD1039B5889411E11EAF2
S315080086A052250ED1002A7FD1A068002800F08480C8
S315080086B0012812D0431C72D0A368A061002B6BD08E
S315080086C0039B227C02F04000C1B2002957D1A06961
S315080086D05969861E8A1E964233D34FF0020884F8DB
S315080086E01180C8E7E2696569B24202D0E06885424E
S315080086F06AD3ED05E661ED0DC5F5007605F12803AB
S31508008700BE4228BF3E4659463246E018FDF7A8FC49
S31508008710217C41F0400222746069D9F80010E368B0
S31508008720321893422CBFE360E2608819BF1B62616E
S31508008730B344C9F80000ABD1217C41F0200323746F
S3150800874099E75889996A06FB0016002EC5D05FEA94
S31508008750572A2E44C6D005EB0A01814288BFC5EBCD
S31508008760000A5946587832465346F8F733FEB0B9E8
S31508008770E069861BB24531D84FEA4A26CCE75878D5
S31508008780E26901990123F8F725FE40B9267C039B87
S3150800879026F0400222749AE7039BA06091E74FF007
S315080087A0010884F8118066E72046A169FEF74AFAAF
S315080087B000287FF47DAFBFE720462946FEF742FA38
S315080087C000287FF475AFB7E7587801993246012338
S315080087D0F8F7D2FD0028E2D165698AE74FF40072FE
S315080087E001980BEB4621FDF73BFC237C23F0400266
S315080087F02274C1E770B50A2982B00E4604461BD01A
S315080088006268002A08DBA318551C3C2D1E7305DC7C
S31508008810A16865604A1CA26002B070BD21462A465E
S3150800882051F80C0B01ABFFF70BFF0198854214BFFB
S315080088304FF0FF350025EBE70D21FFF7DBFFDFE7FC
S3150800884070B582B001A90446FDF7EEFB002845D1B4
S31508008850237C03F02002D1B200293FD003F0400068
S31508008860C3B26BB10199E2694878012304F1280182
S31508008870F8F7B0FD002833D1227C22F0400020749E
S315080088800198216AFDF73CFE40BB636ADD7A45F034
S315080088902006DE72A26821689A76C2F30720D87687
S315080088A00D78032D1ED0E168019D1977080C0E0A74
S315080088B0090E00229877D977612048219A75DA75CA
S315080088C0187659769A74DA745E7701232846EB701F
S315080088D0FDF7AAFD227C22F02001217402B070BDAA
S315080088E00120FBE7160C320A1E755A75DBE700BF36
S315080088F010B582B00446FFF7A3FF08B102B010BD59
S31508008900204601A9FDF790FB0028F7D12060F5E77E
S31508008910F0B583B00D4601A90446FDF785FB06466A
S31508008920002850D1667C002E4DD1E368AB4206D2B2
S31508008930227C02F00200C1B2002908BF1D460023AE
S3150800894062696361002D3ED0019F788947023AB17A
S31508008950013A691EB1FBF7F0B2FBF7F3984260D211
S31508008960A268002A63D0A261002A32D1636915463B
S31508008970D805C10D002965D0E269AA4262D0277CD4
S3150800898007F04003D8B204F1280750B10199012332
S3150800899048783946F8F71EFDC0B9227C22F0400314
S315080089A023740198394640782A460123F8F7E4FCEF
S315080089B060B96369E168E561994204D2227CE360A3
S315080089C042F020002074304603B0F0BD01266674DC
S315080089D0F9E7BD4213D837E0FEF734F90246002816
S315080089E049D0511CF2D0012A18D901994869824206
S315080089F014D26369A261F818AF42606125D2207C5F
S31508008A0000F00203DBB2ED1B20461146002BE3D132
S31508008A1011462046FDF794FD0246E2E702266674F3
S31508008A20D1E779420A406261AD1AA2699CE711460C
S31508008A302046FEF707F901280246EFD00130C5D0D7
S31508008A40A26090E7E168B7E76069E9054319C80DD0
S31508008A50636170B101994869023A02388242DDD2EF
S31508008A604889896A00FB0212002AD7D002EB5525ED
S31508008A707EE705467CE760693D46E6E730B591B096
S31508008A8010AB0D4643F83C0D05A918460022FDF724
S31508008A9051FE044610B1204611B030BD0E4801996A
S31508008AA00F9002AA05A80D92FEF7A2FC044600281C
S31508008AB0F1D10D9991F90B30002B0ADB002DEAD084
S31508008AC0A8750B980028E6D005A82946FDF7E2FA0E
S31508008AD0E1E70624DFE700BF9025002030B59DB00A
S31508008AE01CAB022243F86C0D02A91846FDF722FEBC
S31508008AF002460298069012B110461DB030BD284AAB
S31508008B000199109203AB06A80E93FEF771FC024674
S31508008B100028F1D10E9991F90B00002824DB9DF865
S31508008B201E30DA071ED4029D0D9A2978D47E907ECF
S31508008B30032940EA042405D1507D127D42EA00212A
S31508008B4044EA014403F01003D8B278B906A8FEF740
S31508008B5001FE02460028CFD1D4B90298FDF764FC7D
S31508008B600246C9E70722C7E70622C5E711A800217A
S31508008B7011951394FDF74EFD02460028BCD111A8A5
S31508008B80FEF74AFE02460028ECD00428DED0B3E7FA
S31508008B9006A82146FEF70AFE02460028ACD1DCE705
S31508008BA0902500202DE9F041804682B016464F1EDA
S31508008BB00546002411E0012201AB30466946FFF75D
S31508008BC08BFC019B012B0AD19DF800000D28F2D0E1
S31508008BD001340A2805F8010B01D0BC42EBDB002161
S31508008BE029708C4214BF4046084602B0BDE8F081A1
S31508008BF010B594B0027801910023029303935AB1F9
S31508008C000446114601A8FFF7F5FD14F8012F002ABE
S31508008C10F7D1029A002A0CDB019804A96B46FFF7E4
S31508008C200FFD30B90098029A824202D1039814B017
S31508008C3010BD4FF0FF30FAE77F2830B414D9A9B930
S31508008C400F4B07E05288A9B24C1C824209D0A1B248
S31508008C50802912D05C889A1C4D1C844202F10203BA
S31508008C60F0D101F1800080B230BC7047FF2804D8EB
S31508008C708038044931F81000F6E70020F4E700BF11
S31508008C807EAB000880AB000870B4294E294CB0F5BD
S31508008C90805F28BF2646331D33F8042C1E468AB14A
S31508008CA090420FD333F8021CCCB21519090AA84210
S31508008CB00ADB04330029EFD106EB4406EBE7801AFA
S31508008CC033F8100070BC70470829FBD801A454F883
S31508008CD021F000BFBF8C0008018D00080D8D00082B
S31508008CE0138D0008198D00081F8D0008258D0008B2
S31508008CF02B8D0008F98C0008A0F5E35080B2E1E757
S31508008D00841A04F00102811A88B2DBE7103880B2AF
S31508008D10D8E7203880B2D5E7303880B2D2E71A389B
S31508008D2080B2CFE7083080B2CCE7503880B2C9E7C6
S31508008D3080AC0008C4AA0008013A70B48D18A9428C
S31508008D403ED24B780A7803EB022293B2C018CA4384
S31508008D5080B2AA188342C2F3400235D88B1C9D42C2
S31508008D6028D96AB11C785A7802EB042292B2801884
S31508008D7080B2824201D9421C90B202339D4219D96F
S31508008D801E785C7804EB0624A4B2001980B29A1CFB
S31508008D90844201D9441CA0B29C78537803EB04237F
S31508008DA09BB2C01880B2834201D9431C98B2931C67
S31508008DB09D42E5D8CA43AB1823F00102931CC91893
S31508008DC0A94204D070BC7047431C98B2C6E709781C
S31508008DD00A02101880B28242F4D9431C98B2F1E70D
S31508008DE038B50E4C657C237C143D05EB03218DB20A
S31508008DF0401904F11A01082280B2FFF79DFF04F119
S31508008E0022012A46FFF798FF10B94FF6FF7038BDC2
S31508008E10020A42EA002398B238BD00BF142800208F
S31508008E2070B4C478134B0A19D4B2DC7086780D0A6C
S31508008E30AA19D2B29A7046785E7000789542187070
S31508008E4003D90136F6B25E708EB1C9B28C420CDA1D
S31508008E500132D0B20749987038B94B785A1CD0B24B
S31508008E60487010B90B785A1C0A7070BC70470130EC
S31508008E701870EAE7682E002010B5094C23680146E9
S31508008E8003F10800FFF7CCFF064A236850781478E8
S31508008E909178D2781C7258729972DA7210BD00BF36
S31508008EA098270020682E002008B5002006491422BD
S31508008EB0FFF742FF10B94FF6FF7008BD030A43EAF1
S31508008EC0002080B208BD00BF222800200620FFF738
S31508008ED087BF00BF42F67C6042F29C71C2F2000076
S31508008EE0C2F2000142F6786242F66C6330B4C2F20E
S31508008EF000020024C2F2000304804C7601204FF4DD
S31508008F00806125461070198030BC7047064B074AA9
S31508008F10198810B40024147019B10120107010BCFF
S31508008F2070471880FBE700BF7C2E0020782E0020B3
S31508008F302DE9F04FB74CB84AB84FB94BD2F8009064
S31508008F4004F1360103288BB0396019600DD0022868
S31508008F501AD0A07B452800F0C780B24EB24D00203B
S31508008F60288030700BB0BDE8F08F99F8195005F0DD
S31508008F700F06032EF1D1B9F81000AA4EAA4D002803
S31508008F80EDD1DFF8B0822EE0A84DEE78711CC8B29C
S31508008F90E87060B9AA78561CF1B2A97039B9687830
S31508008FA0421CD6B26E7016B92978481C287099F8F2
S31508008FB019209D4DDFF87C820026072A2E80A8F806
S31508008FC0006000F0E080052A00F0DD80002A00F04D
S31508008FD0E380B9F81010002940F0E08002F00F0095
S31508008FE00328904EBBD108223270009301F040F955
S31508008FF0009B327802F02001C9B2002900F06A818C
S315080090000021A8F800101420DFF82C8289F819101E
S3150800901084F82F0028222A80502784F82E7099F881
S315080090200810B8F8007084F82A1099F80930B8F8CA
S31508009030021084F82B3099F80A00764B84F82C0035
S3150800904099F80B2084F82D2099F80C0084F826004E
S3150800905099F80D2084F8272099F80E0084F828003E
S3150800906099F80F00062284F82900E275B9F8040079
S315080090706084B9F806006783A084A183B9F8001054
S31508009080E183B9F80200208499F8191001F010005C
S31508009090C1B2002900F00C81002083F8310083F862
S315080090A030002B88402100251A0AA17522746374A2
S315080090B084F8355084F834506586FFF707FF5C4A14
S315080090C0E57313886575591C8BB2C043190A608607
S315080090D045201380A0732575A174E3742583FFF7D3
S315080090E0E3FEC24322834BE04F4D94F81090667C12
S315080090F0298806EB092989454EDC207D1FFA89F95E
S315080091008006A5F8009047D1667D002E44D1DFF889
S315080091102881B8F80060002E40F0D080B8F8021018
S31508009120002940F0CB8001920093FFF7BDFE4FF671
S31508009130FF7290428246009B01982DD1E17DDFF8AF
S31508009140D4B0062900F01A81012925D19BF82220DE
S31508009150082A21D1BBF824004FF6F671002388426D
S315080091608BF8223040F29E810930ABF82400608BE0
S31508009170A28BB8F8023066832A4EE0832284A38342
S3150800918000233370EEE699F81A60701CC2B2782A8A
S3150800919089F81A2000F08780224EE0E699F81A60CE
S315080091A0711E89F81A10002EF6D199F81B60082E40
S315080091B000F0CF80501E012840F2C880042E00F22D
S315080091C0C180032101FA06F1C8B202F00F02013686
S315080091D0511E89F81A0089F81B600729DCD801A0F6
S315080091E050F821F09F9200086F9200083D920008FF
S315080091F005920008999100080592000899910008BF
S3150800920005920008074EDFF83080112384F82F30C6
S3150800921000E700BF1428002098270020582E0020B9
S31508009220802E0020642E0020082800205C2E0020B6
S315080092300A28002010280020602E0020C24E042094
S315080092403070009301F014F8B8F80020009B1B68F2
S315080092503B60002A67D0B9F81000002863D0283090
S315080092601823288084F82F30DFF8F482D4E6DFF854
S31508009270F0820227042684F82F70022206210A2388
S315080092802C20602784F8376084F8362084F8381054
S3150800929084F83930288084F82E70AB4EBFE6DFF8A4
S315080092A0C0821227E6E7002189F81910A64E56E66D
S315080092B083F830200A2283F83120F2E6E08BB042A8
S315080092C07FF46AAFA149088CB8F8021088427FF487
S315080092D063AF28E702F01000C0B278B1012004227B
S315080092E01127A9F8100089F8192089F81B10A8F881
S315080092F0001084F82F70DFF868828BE6B8F8001043
S3150800930011B3D20733D5A9F81000B9F81220914243
S3150800931088BFA8F80020B8F80020A9F81020002176
S3150800932089F81B1093E7327802F00201CBB2002BC2
S315080093303FF415AE282710212F8084F82F10DFF868
S31508009340208269E6302040E70A46E8E7052E7FF4E2
S3150800935035AF00227C4E89F819208021317000F043
S3150800936087FF142384F82F30DFF8F48152E6B9F822
S315080093701020002AC9D076480280D0E700930190D1
S31508009380FFF7A4FD5045019A009B7FF405AFDFF86F
S31508009390D4A19AF8190030B1BBF82460BAF80410C1
S315080093A08E4200F0838094F82F3003F03F06022E99
S315080093B05ED0654E94F82F20644B02F00400C1B2CB
S315080093C000297FF4CCAD93F82DA093F82BC093F821
S315080093D0297083F829A04FF0140A93F8262093F8E9
S315080093E0280093F82C9093F8271093F82AE083F82E
S315080093F02FA001374FF0280A83F827C0DFF85CC191
S31508009400A5F800A0FFB24FF0500A83F82EA083F803
S31508009410289083F82C0083F82B108CF8002083F80A
S3150800942026E083F82A2083F82D7067B90130C7B281
S3150800943083F82C703FB90131C8B283F82B0010B9F4
S31508009440013283F82A20638CB4F824E0678BB4F8D9
S315080094501CC0B8F80010B8F802203E48A4F822E06C
S315080094600380A384E783A4F820C06183A28318E657
S31508009470364F3949BB8C0988DFF8D890374FA9F899
S315080094800030002699423E7003D001222E4E3A70D3
S3150800949090E7002800F02381072800F01E810120AC
S315080094A0387079E60830ABF8240060E6BBF822602D
S315080094B0BAF806108E427FF476AFBBF81A60BAF88F
S315080094C000108E427FF46FAFBBF81C60BAF802102A
S315080094D08E427FF468AF9BF82FC01B4ECDF808C0AC
S315080094E00CF0040E00215FFA8EFCC2F800A0317061
S315080094F0BCF1000F66D19BF82EE0DFF860B04FEAAA
S315080095001E1C4FEA8C01A9F11409C1EB090E00F0E3
S315080095100F001FFA8EF902288BF80010A5F80090A4
S3150800952022D0B9F1000F02D10298810722D0B4F8EF
S3150800953026E0BAF808108E4558D01027DFF8249090
S3150800954084F82F7066E500BF642E002014280020DA
S31508009550102800206E2E00207C2E0020782E002059
S31508009560602E00209C270020DDF808C00CF03F0183
S315080095701229D6D1DDF808E00EF01001C8B220B1E4
S31508009580BAF81010DFF84893C1BB9AF8191001F021
S315080095900F00013807283FF6E2AC0FF2080C5CF81A
S315080095A020F000BFAB990008859900087598000857
S315080095B039980008E3970008CB9700083B95000800
S315080095C0D395000820228AF81910327000F050FE50
S315080095D0C5E43378DB077FF5C2AC0022BA488AF8BF
S315080095E019201021017000F043FEB8E4B748B849C5
S315080095F0B0F828C0488984459FD1BBE709F10C001B
S3150800960001920093FFF70CFCB24994F82A2091F8CE
S3150800961000C0009BCDF808C09445019AB5D142F622
S315080096201400C2F2000091F801E090F82B00CDF882
S315080096300CE08645A9D142F61400C2F2000091F862
S3150800964002C090F82C00CDF814C084459DD142F68E
S315080096501400C2F20000C97890F82D00814294D116
S31508009660DDF808E0DDF80CC089F80CE099F81B0075
S31508009670DDF814E089F80DC089F80EE089F80F10B6
S3150800968008BB99F818C099F81A0099F81610C0EB93
S315080096900C00A0EBD100C0B241185FFA81FEC1B23E
S315080096A011F0800F89F816E001D04042C1B29AF84D
S315080096B01700A0EB90004118C8B200EBDE0C8AF840
S315080096C017008AF818C09AF8181001208AF81A1094
S315080096D000213070AAF8101057E7012139707E4E24
S315080096E0C2F800A096F800C096F801E0B178F078C4
S315080096F094F82960AAF80430069694F8276005902D
S315080097004FF0030B8AF81AB08AF818B008964FF08B
S31508009710040B00268AF816608AF817B08AF81B60C8
S31508009720638C94F82800AAF80630638B0790AAF889
S31508009730003094F82600A38B8AF80CC08AF80E101D
S31508009740DDF814C00699099001221046AAF80230DD
S315080097508AF819208AF80DE08AF80FC0AAF81020AE
S315080097608AF80B10079ADDF820E0099B8AF80A2088
S315080097708AF809E08AF80830FFF77EFB94F82E008D
S3150800978000F0F001502940F34D8120FA0BF3534ABB
S31508009790581F800013780EE091F836307BB1012B04
S315080097A000F04481022B2BD09EF8371001EB060EF1
S315080097B029B15FFA8EF6A11986428E46ECDB3E7019
S315080097C01370DFF80C91122754E53378DB077FF521
S315080097D0C6AB072200218AF819208AF81A10FFF763
S315080097E0BEBB288808B1FFF747FB94F82F00C207CD
S315080097F000F11F812A88002A7FF49FAEFFF7AFBBCE
S3150800980091F837C0BCF1040FCED191F8380091F821
S315080098103910137041EA002203F5C1639A4238BF32
S3150800982013463E70A9F80020AAF81230AAF8143098
S31508009830DFF89C9012271DE5288808B1FFF71CFB66
S3150800984094F82F1011F0010000F091803778F8078E
S3150800985040F18980002307228AF819208AF81A30ED
S31508009860AAF810300120FFF707FB1021317000F02D
S31508009870FFFC62E694F82F20D00731D501F01000DE
S31508009880C0B268BBBAF81030002B7FF468AB2F88DB
S31508009890791C88B2FFF7F0FA30782A8840F010036E
S315080098A033701AB1084940F012070F7000F0E0FC57
S315080098B0012008220023DFF81890AAF810008AF879
S315080098C019208AF81B30A0E4642E002014280020F2
S315080098D09C270020682E00205C2E0020842E002065
S315080098E002F02002D0B268B194F8348094F83500BA
S315080098F03A68B5F800E040EA08201218C0EB0E00F6
S315080099003A602880288858B101F01001CAB23AB9DD
S31508009910317841F0020232700093FFF7ADFA009BEE
S3150800992094F830C094F83110BAF814006C4A01EB78
S315080099300C2189B28142118000D801B910801088A3
S315080099403278AAF8120091073FF409ABDFF8A08134
S31508009950DFF8A0910020A8F80000009300F088FC2A
S31508009960009BFFF746BB06208AF819007AE733788A
S31508009970D9077FF53FAF05218AF81910AAF8100014
S31508009980FFF7EDBA3178C90705D594F82F0000F02E
S315080099903F01122920D020233370019200F068FC81
S315080099A0019A10680021417604E531784D4AC807C6
S315080099B07FF5D5AA03218AF8191028884021117045
S315080099C00021AAF810100028C0D042211170009377
S315080099D0FFF752FA009BB9E7434991F82E2002F0A7
S315080099E0F00050284CDD41481109A1F1050801781D
S315080099F04FEA880C002204EB020E6245F04668DA4C
S31508009A009EF83610002964D0012966D002291ED096
S31508009A1098F837E00EEB0208BEF1000F59D05FFA4E
S31508009A2088F2E8E7DFF8CC90122723E40136F6B28D
S31508009A30C1E60023072701208AF819708AF81A3028
S31508009A40FFF71AFA1022327000F012FC75E59EF83C
S31508009A503790B9F1040FDBD19EF838C09EF83990DB
S31508009A6001708BF8002049EA0C2001F5C1611C4AF7
S31508009A70884238BF01461080AAF81210AAF81410B6
S31508009A8094F8260094F827E094F8281094F82920EA
S31508009A908AF808004FF0030C8AF819C08AF809E01A
S31508009AA08AF80A108AF80B2001200093DFF8408014
S31508009AB0DFF84090FFF7E0F900234220AAF81030BB
S31508009AC02B80A8F80030307000F0D2FB009BFFF71F
S31508009AD090BA01708BF80020D2E70132D2B28AE739
S31508009AE06E2E0020642E002014280020842E0020CC
S31508009AF0102800209C270020030A43EA002080B291
S31508009B00704700BF0A1E034609DD0549086805496E
S31508009B1083420A8003D0194692B200F0EFBB704721
S31508009B20802E002010280020F8B59C4B9C4A1888E7
S31508009B309C4E918BD48B20B15A8812B1884200F082
S31508009B40DA809A89954822B1C58915B18A4200F00A
S31508009B50ED801A8B914822B1458B15B18A4200F0E7
S31508009B60EC809A8C8D4822B1C58C15B18A4200F0DA
S31508009B70EB801A8E894822B1458E15B18A4200F0CB
S31508009B80EA809A8F854822B1C58F15B18A4200F0BE
S31508009B90C680B3F8482081482AB1B0F84A5015B1B2
S31508009BA08A4200F0AE80B3F854207C482AB1B0F857
S31508009BB0565015B18A4200F0AB801D88774C1DB906
S31508009BC06588002D00F094809989744C19B9E2894A
S31508009BD0002A00F0D080188B704C18B9658B002DC0
S31508009BE000F0CC80998C6D4C19B9E28C002A00F0F3
S31508009BF0C880188E694C18B9658E002D00F0C4808F
S31508009C00998F664C19B9E28F002A00F0C080B3F824
S31508009C104800624C20B9B4F84A50002D00F0BA80CA
S31508009C20B3F854105D4C00295CD05F4D9F7A2978B3
S31508009C300024CF1B22462046A7429C7DC8BFFAB205
S31508009C400C1B9442C8BFE2B293F82240C4EB01044D
S31508009C50C8BF01209442C8BFE2B293F82E40C4EBB5
S31508009C600104C8BF02209442C8BFE2B293F83A4042
S31508009C70C4EB0104C8BF03209442C8BFE2B293F8FC
S31508009C804640C4EB0104C8BF04209442C8BFE2B2F0
S31508009C9093F85240C4EB0104C8BF05209442C8BFDC
S31508009CA0E2B293F85E40C4EB0101C8BF06209142B8
S31508009CB0C8BFCAB23D49C8BF07200A703C4A3070BF
S31508009CC000EB4004107003EB84043A490422204652
S31508009CD000F014FB201D3849062200F00FFB2B78F4
S31508009CE0A372F8BDB4F85620002A9ED1072554342D
S31508009CF035702D4DE9E7A2427FF423AF00221C46BA
S31508009D002FE0A5427FF44FAF062200F1480428E071
S31508009D10A5427FF452AF072200F1540421E0A54280
S31508009D207FF437AF052200F13C041AE0A5427FF420
S31508009D3010AF012200F10C0413E0A5427FF411AF25
S31508009D40022200F118040CE0A5427FF412AF0322A8
S31508009D5000F1240405E0A5427FF413AF042200F1C4
S31508009D60300415493270201D062200F0C7FA0E4845
S31508009D700178A172F8BD01250C34B9E7022518341B
S31508009D80B6E703252434B3E704253034B0E70525C0
S31508009D903C34ADE706254834AAE700BF882E0020E4
S31508009DA014280020852E0020E92E0020862E00206B
S31508009DB0E82E0020302800202A28002070B5154EED
S31508009DC0154C3278154D0023501C3070237005E071
S31508009DD02078421CD3B2072B23701AD803EB43030F
S31508009DE005EB830035F82310428842EA010399B24D
S31508009DF00029EDD03278837AD11A7729E8DD042252
S31508009E00002100F09FFA2078421CD3B2072B23705A
S31508009E10E4D970BDE92E0020852E0020882E00206A
S31508009E20F8B52A4C2388292B40D9294DAA8A00201F
S31508009E30B2F5807F2080074603D0B2F5007F38D080
S31508009E40F8BD244EE98C32889142F9D1288D738861
S31508009E509842F5D1FFF768FE022305F1160106229E
S31508009E6005F120006B752F7500F048FA1A4906228D
S31508009E7005F1160000F042FA06221749A81800F064
S31508009E803DFA05F120010622284600F037FAA88B8C
S31508009E90E98B32887388E8842985AA8308200621F5
S31508009EA02A22EB83287369732280F8BD0023238056
S31508009EB0F8BD084BE98C1A889142C1D1288D5B8878
S31508009EC09842BDD1BDE8F840FFF72EBE082800200D
S31508009ED014280020602E0020702E0020F8B56F4C44
S31508009EE0E38B4FF6FF7293427AD06D4E6D4D3288F2
S31508009EF0298883EA0200084267D06B496B4D0B88B4
S31508009F0048882B8068806A4ADFF8C8E11088698823
S31508009F1098427BD09089664F984200F08480108BD7
S31508009F20634F984200F08F80908C614F984200F002
S31508009F308280108E5E4F984200F08D80908F5C4F25
S31508009F40984200F09080B2F84800594F984200F0C5
S31508009F509B80B2F8542056489A4200F08C80082715
S31508009F60FF2106224D488EF8007000F0EBF900211B
S31508009F700622504800F0E6F94F495048062200F0FC
S31508009F80BDF94D494E48062200F0B8F9298870886F
S31508009F90E18400230121E0830420B5F802C0E074BF
S31508009FA0062223756175A373E17363743588454981
S31508009FB0454B46486273A2742A2227742773A4F86D
S31508009FC028C0A58319600280F8BD218C70886D8829
S31508009FD081EA00022A4290D1344D2B80698092E7AB
S31508009FE0208C984281D120463949062200F086F90C
S31508009FF031493248062200F081F93448028808239C
S3150800A0000E320021237361730280F8BD508888429E
S3150800A01080D1002311460431062220488EF80030EC
S3150800A02000F06CF9E4E7F88988427FF478AF0123F9
S3150800A03007F10C01EFE7F88C88427FF47AAF032327
S3150800A04007F12401E7E7788B88427FF46DAF022396
S3150800A05007F11801DFE7788E88427FF46FAF042393
S3150800A06007F13001D7E7F88F88427FF46CAF0523F4
S3150800A07007F13C01CFE7B0F856308B427FF46FAF5B
S3150800A080072300F15401C6E7B7F84A0088427FF46F
S3150800A09060AF062307F14801BDE700BF142800207A
S3150800A0A0602E0020042800200C280020EC2E00201A
S3150800A0B0882E002034280020702E00201A28002020
S3150800A0C02A2800204A280020582E00200828002088
S3150800A0D074AE0008852E002038B5F8F741F8FAF76F
S3150800A0E0A5FD42F6F463C2F2000300F5FA701860A3
S3150800A0F0FAF79CFD42F6F061C2F2000100F51C5227
S3150800A10010320A60FEF7E6FE42F66061C2F200010E
S3150800A11042F60402C2F200024FF6A96443F613752A
S3150800A1200C804D8042F60C034FF6FF71C2F2000315
S3150800A1301180002151804EF6030040F213121C8054
S3150800A1405A80FEF7E3FEBDE83840F8F737B900BF96
S3150800A150F8B5164B1F68FA693A62E1B14C1EA4B20B
S3150800A160661C012307F11C020578B342157204EA3E
S3150800A170030410D02CB144780223B34287F8254053
S3150800A18009D0C55CD41801332572C55CD4180133CF
S3150800A190B3422572F5D10431A7F8641007F12000FF
S3150800A1A0FFF7B0FCF869411CF961F8BD9827002053
S3150800A1B070B5F8F715F9F8B9FAF738FD264B1A68A5
S3150800A1C090420BD325482649264C086002F5FA72B8
S3150800A1D002201A60FEF7ACFE238843BBFAF726FD79
S3150800A1E021490A68904205D302F51C5310330B60C7
S3150800A1F0FFF7E4FD002070BD1A4D1C4C28804FF473
S3150800A2000060A689FFF778FC864217D040F606005C
S3150800A210A489FFF771FC8442CED1FFF701FE2B8893
S3150800A220002BC9D0F8F700F900202880C4E7FFF70B
S3150800A23055FEF8F7F9F800202080CFE70120FEF751
S3150800A24077FE29880029B7D0FFF748FEF8F7ECF81B
S3150800A25000222A80B0E700BFF42E00209C270020A9
S3150800A2609827002008280020F02E00201428002017
S3150800A27038B5174D174A2B78146803F04000C2B258
S3150800A280CAB9D90703F00401C8B248BFA4F86420C4
S3150800A29010B1B4F86410A1B903F00202D1B201B941
S3150800A2A038BD0D4802680023101DA4F86430BDE8C7
S3150800A2B03840FBF70DB901210020E161A4F86400DC
S3150800A2C038BD04F12000FFF71DFC2B78E4E700BF3A
S3150800A2D0642E002098270020582E0020A0F1300078
S3150800A2E009288CBF00200120704700BFA0F1610338
S3150800A2F0D9B2192998BF2038704700BF844640EA6A
S3150800A300010313F0030F40F01080242AC0F00D80DB
S3150800A3102DE9F00FB1E8F80FA0E8F80FA2F1240232
S3150800A320242ABFF4F7AFBDE8F00F002A00F0078033
S3150800A33011F8013B00F8013B013A7FF4F9AF60469A
S3150800A340704700BF8446002A00F0328010F0030FE1
S3150800A35000F0078000F8011B013A00F02980FFF79A
S3150800A360F5BF282AC0F01F80A2F128022DE9F00FB8
S3150800A37001F0FF0141EA012141EA014141EA016197
S3150800A3800B460C460D460E460F46884689468A46B3
S3150800A3908B46A0E8FA0F283ABFF4FBAFBDE8F00FEA
S3150800A3A0283200F0058000F8011B013A7FF4FBAF64
S3150800A3B06046704738B504460D4600F019F842F66F
S3150800A3C0F863C2F200031D6044F0800442F6FC60A4
S3150800A3D0C2F200000460024611680029FCD100F0B0
S3150800A3E009F842F6F863C2F20003186838BD00BFE0
S30D0800A3F0704700BF704700BF6B
S3150800A3F8433A2F55736572732F766F6F726275724B
S3150800A408672F4465736B746F702F426C7454657349
S3150800A418742F5461726765742F44656D6F2F4152A6
S3150800A4284D434D345F53544D333246345F4F6C6950
S3150800A4386D65785F53544D3332453430375F437210
S3150800A4486F7373776F726B732F426F6F742F6964AC
S3150800A458652F2E2E2F6C69622F7569702F6E65749D
S3150800A4686465762E63000000020102002F64656D9C
S3150800A4786F70726F675F6F6C696D65785F73746DFF
S3150800A4883332653430372E73726563002F626F6F07
S3150800A498746C6F672E7478740000000057696E55DF
S3150800A4A853422042756C6B20496E74657266616307
S3150800A4B86500000044656661756C7400303030309C
S3150800A4C83030303030353043000000004F70656E4C
S3150800A4D8424C5420557365720000000057696E5542
S3150800A4E853422042756C6B204465766963650000A3
S3150800A4F8433A2F55736572732F766F6F726275724A
S3150800A508672F4465736B746F702F426C7454657348
S3150800A518742F5461726765742F44656D6F2F4152A5
S3150800A5284D434D345F53544D333246345F4F6C694F
S3150800A5386D65785F53544D3332453430375F43720F
S3150800A5486F7373776F726B732F426F6F742F6964AB
S3150800A558652F2E2E2F2E2E2F2E2E2F2E2E2F536F63
S3150800A568757263652F41524D434D345F53544D33CD
S3150800A5783246342F43726F7373776F726B732F7605
S3150800A5886563746F72732E6300000000433A2F5593
S3150800A598736572732F766F6F72627572672F44656B
S3150800A5A8736B746F702F426C74546573742F54618F
S3150800A5B8726765742F44656D6F2F41524D434D344C
S3150800A5C85F53544D333246345F4F6C696D65785F17
S3150800A5D853544D3332453430375F43726F7373774C
S3150800A5E86F726B732F426F6F742F6964652F2E2EE7
S3150800A5F82F2E2E2F2E2E2F2E2E2F536F7572636504
S3150800A6082F41524D434D345F53544D333246342F00
S3150800A61863616E2E6300000005020602060307033F
S3150800A6280803090309040A040B040C040C050D05A0
S3150800A6380E050F050F06100610071008000008007B
S3150800A6481000180020002800300038004000480094
S3150800A658500058008000880090009800A000A800C4
S3150800A668B000B800C000C800D000D80000C0000874
S3150800A6780040000003000000000001080000010077
S3150800A688040000000000020800000200050000009F
S3150800A6980000040800000200060000000000060882
S3150800A6A80000020007000000000008080000020079
S3150800A6B80800000000000A0800000200090000005F
S3150800A6C800000C08000002000A00000000000E083E
S3150800A6D8000002000B000000433A2F557365727399
S3150800A6E82F766F6F72627572672F4465736B746F16
S3150800A6F8702F426C74546573742F5461726765744D
S3150800A7082F44656D6F2F41524D434D345F53544D59
S3150800A718333246345F4F6C696D65785F53544D33F1
S3150800A72832453430375F43726F7373776F726B7362
S3150800A7382F426F6F742F6964652F2E2E2F2E2E2F9A
S3150800A7482E2E2F2E2E2F536F757263652F41524D5D
S3150800A758434D345F53544D333246342F7561727402
S3150800A7682E630000433A2F55736572732F766F6F01
S3150800A77872627572672F4465736B746F702F426CBB
S3150800A78874546573742F5461726765742F44656DC4
S3150800A7986F2F41524D434D345F53544D333246342F
S3150800A7A85F4F6C696D65785F53544D333245343065
S3150800A7B8375F43726F7373776F726B732F426F6F5E
S3150800A7C8742F6964652F2E2E2F2E2E2F2E2E2F2EA0
S3150800A7D82E2F536F757263652F41524D434D345F63
S3150800A7E853544D333246342F7573622E6300000076
S3150800A7F808003F0008003F004F70656E424C540041
S3150800A808303A0000433A2F55736572732F766F6F87
S3150800A81872627572672F4465736B746F702F426C1A
S3150800A82874546573742F5461726765742F44656D23
S3150800A8386F2F41524D434D345F53544D333246348E
S3150800A8485F4F6C696D65785F53544D3332453430C4
S3150800A858375F43726F7373776F726B732F426F6FBD
S3150800A868742F6964652F2E2E2F2E2E2F2E2E2F2EFF
S3150800A8782E2F536F757263652F66696C652E630094
S3150800A8884669726D776172652075706461746520B2
S3150800A8987265717565737420646574656374656437
S3150800A8A80A0D00004F70656E696E67206669726DDD
S3150800A8B8776172652066696C6520666F72207265B5
S3150800A8C86164696E672E2E2E000000004552524FAD
S3150800A8D8520A0D004F4B0A0D0000000053746172AE
S3150800A8E874696E67207468652070726F6772616D27
S3150800A8F86D696E672073657175656E63650A0D0007
S3150800A90850617273696E67206669726D77617265E0
S3150800A9182066696C6520746F2064657465637420A5
S3150800A928657261736520626C6F636B732E2E2E00D9
S3150800A93845726173696E67200000000020627974A9
S3150800A94865732066726F6D206D656D6F727920610B
S3150800A958742030780000000052656164696E6720CB
S3150800A9686C696E652066726F6D2066696C652E2E39
S3150800A9782E4552524F520A0D00000000496E766164
S3150800A9886C696420636865636B73756D20666F759B
S3150800A9986E642E2E2E4552524F520A0D00000000A4
S3150800A9A850726F6772616D6D696E672000000000EE
S3150800A9B820627974657320746F206D656D6F72797E
S3150800A9C8206174203078000057726974696E6720B0
S3150800A9D870726F6772616D20636865636B73756DF6
S3150800A9E82E2E2E00436C6F73696E67206669726D2A
S3150800A9F8776172652066696C650A0D004669726D2D
S3150800AA087761726520757064617465207375636310
S3150800AA1865737366756C6C7920636F6D706C657495
S3150800AA2865640A0D00000000222A3A3C3E3F7C7FF6
S3150800AA38000000002B2C3B3D5B5D0000809A4541D9
S3150800AA488E418F804545454949498E8F9092924F48
S3150800AA58994F555559999A9B9C9D9E9F41494F5583
S3150800AA68A5A5A6A7A8A9AAABACADAEAFB0B1B2B317
S3150800AA78B4B5B6B7B8B9BABBBCBDBEBFC0C1C2C308
S3150800AA88C4C5C6C7C8C9CACBCCCDCECFD0D1D2D3F8
S3150800AA98D4D5D6D7D8D9DADBDCDDDEDFE0E1E2E3E8
S3150800AAA8E4E5E6E7E8E9EAEBECEDEEEFF0F1F2F3D8
S3150800AAB8F4F5F6F7F8F9FAFBFCFDFEFF7D1D010033
S3150800AAC8632C001E9601A01E5A01001F0806101FB7
S3150800AAD80606201F0806301F0806401F0606511FCF
S3150800AAE80700591F521F5B1F541F5D1F561F5F1F04
S3150800AAF8601F0806701F0E00BA1FBB1FC81FC91F94
S3150800AB08CA1FCB1FDA1FDB1FF81FF91FEA1FEB1F27
S3150800AB18FA1FFB1F801F0806901F0806A01F0806B5
S3150800AB28B01F0400B81FB91FB21FBC1FCC1F0100F5
S3150800AB38C31FD01F0206E01F0206E51F0100EC1F0F
S3150800AB48F21F0100FC1F4E2101003221702110025C
S3150800AB58842101008321D0241A05302C2F04602C67
S3150800AB680201672C0601752C0201802C6401002D50
S3150800AB78260841FF1A030000C700FC00E900E200A6
S3150800AB88E400E000E500E700EA00EB00E800EF0073
S3150800AB98EE00EC00C400C500C900E600C600F400D3
S3150800ABA8F600F200FB00F900FF00D600DC00A20060
S3150800ABB8A300A500A7209201E100ED00F300FA0022
S3150800ABC8F100D100AA00BA00BF001023AC00BD00EE
S3150800ABD8BC00A100AB00BB00912592259325022550
S3150800ABE8242561256225562555256325512557258A
S3150800ABF85D255C255B251025142534252C251C2563
S3150800AC0800253C255E255F255A2554256925662590
S3150800AC18602550256C2567256825642565255925E9
S3150800AC285825522553256B256A2518250C25882568
S3150800AC3884258C2590258025B103DF009303C0035E
S3150800AC48A303C303B500C403A6039803A903B4035F
S3150800AC581E22C603B50329226122B1006522642291
S3150800AC6820232123F7004822B0001922B7001A2208
S3150800AC787F20B200A025A00061001A03E000170390
S3150800AC88F8000703FF0001007801000130013201CE
S3150800AC980601390110014A012E01790106018001D0
S3150800ACA84D004302810182018201840184018601E3
S3150800ACB88701870189018A018B018B018D018E0124
S3150800ACC88F0190019101910193019401F601960172
S3150800ACD89701980198013D029B019C019D0120025C
S3150800ACE89F01A001A001A201A201A401A401A60135
S3150800ACF8A701A701A901AA01AB01AC01AC01AE01E4
S3150800AD08AF01AF01B101B201B301B301B501B50194
S3150800AD18B701B801B801BA01BB01BC01BC01BE0143
S3150800AD28F701C001C101C201C301C401C501C401BB
S3150800AD38C701C801C701CA01CB01CA01CD01100163
S3150800AD48DD0101008E01DE011201F3010300F101A4
S3150800AD58F401F401F8012801220212013A02090055
S3150800AD68652C3B023B023D02662C3F02400241022B
S3150800AD78410246020A015302400081018601550232
S3150800AD8889018A0158028F015A0290015C025D0204
S3150800AD985E025F029301610262029401640265021F
S3150800ADA866026702970196016A02622C6C026D02B6
S3150800ADB86E029C01700271029D01730274029F0162
S3150800ADC876027702780279027A027B027C02642C80
S3150800ADD87E027F02A60181028202A90184028502F7
S3150800ADE886028702AE014402B101B20145028D020C
S3150800ADF88E028F0290029102B7017B030300FD03BE
S3150800AE08FE03FF03AC0304008603880389038A0349
S3150800AE18B1031103C2030200A303A303C40308036F
S3150800AE28CC0303008C038E038F03D8031801F2039F
S3150800AE380A00F903F303F403F503F603F703F70324
S3150800AE48F903FA03FA0330042003500410076004D0
S3150800AE5822018A043601C1040E01CF040100C00488
S3150800AE68D00444016105260400000000FFFFFFFF27
S3090800AE78FFFF0000CA
S3150800AE7C01000000010000000000000001020304AC
S3150800AE8C01020304060708091C00002051260008C5
S3150800AE9C9525000849250008B1240008192500083D
S3150800AEAC952400087D240008C1240008D124000834
S3150800AEBCE1240008F924000809022000010100C059
S3150800AECC320904000002FF00000007058102400059
S3150800AEDCFF070501024000FF9D4100088541000857
S3150800AEECCD41000800000000000000006D4100087C
S3150800AEFC79410008554100080000000000000000D8
S3150800AF0C454100084542000855420008C54200085C
S3150800AF1CE5420008A542000885420008654200087B
S3150800AF2C040309041201100100000040501DAC6016
S3150800AF3C000101020301000005430008094300084B
S3150800AF4C0D4300082543000821430008194300084F
S30A0800AF5C114300080482
S7050800018968
